:1000000002624E0265830000000000025EB3000041
:100010000000000265E10000000000320000000066
:10002000000000022BD30000000000025FE9000086
:1000300000000000000000000000000000000000C0
:100040005052343032207665722E3132382E342EB2
:1000500032204864773A482030322D30382D303500
:100060002030303A3133202075F00612011E221262
:100070005C2975F00612011E125C2E2212006F120E
:10008000006812006F12006812006F120068120000
:100090006F12006812006F75F01812011E22125CB8
:1000A0002975F04B12011E125C2E22755004122588
:1000B000971225AD125C2975F0C812011E125C2E34
:1000C000227550051225971225AD12009E75F01E5F
:1000D00012011E12009E227550071225971225AD9F
:1000E000120088227550061225971225AD12008E37
:1000F0002212007C12007C221200E41200E41200A2
:10010000E422C2A1C25812006F75F01212011ED271
:10011000A1C2582212006F75F01212011E22128124
:10012000FE201A07C0F012808DD0F0D5F0F02270BA
:1001300004A243B322C0E01412013ED0E022C0E08A
:10014000030303540F28F8D0E0C0E0540704F5F08F
:10015000E213D5F0FCD0E0227003D3802830E7030F
:10016000C3802223F9C3137004A243801814C0E093
:10017000030303540F247AF8D0E0540704F5F0E2A7
:1001800013D5F0FCE992E022C0E024B5F8E21201B8
:10019000584004D0E0C322D0E024CBF58274003470
:1001A00000F583E01201A82220E702C322C2E7C0C3
:1001B000E0C2E0700AA243B3D0E030E001B322B461
:1001C0007E03C380F3B40204A22780ECB40404A22B
:1001D0002880E5B40604A22980DEB40804A20380C6
:1001E000D7B40A04A20E80D0B40C0AE5754576C3D4
:1001F0006001D380C3B40E05125E9580BBB41007B6
:10020000A25E725DB380B1B41206A25D822A80A89C
:10021000B41406A25DB02A809FB41604A25E809832
:10022000B418077400126BB6808EB41A07740112EA
:100230006BB68084B41C087402126BB60201B8B4A9
:100240001E087403126BB60201B8B42008740412BD
:100250006BB60201B8B422087405126BB60201B87D
:10026000B424087406126BB60201B8B426087407E9
:10027000126BB60201B8D0E0C32212317FE56C6088
:1002800013B401051202AC8008B402051202C28048
:1002900000756C0012808DE5775440600B20A80833
:1002A000305505C255128101126A0B22C2437518DE
:1002B0006075190F751AFA120A37757E03C245C2A6
:1002C0004822D24375187075190F751AFA120A3739
:1002D000757E0322C2B612652C753700740312476F
:1002E00005E51E124705E51F12470574571247051D
:1002F0001202FDE5371247053099FDD3227884E6D6
:10030000232354031247057885E630E402240A5477
:100310000F1247057884E6C4540375F00AA4F5F07B
:10032000E6540F25F01247057883E6C4540375F0B0
:100330000AA4F5F0E6540F25F01247057882E6C4CA
:10034000540775F00AA4F5F0E6540F25F01247059E
:100350007881E6C4540775F00AA4F5F0E6540F2539
:10036000F01247057885E603C45407124705227545
:10037000F032128216B2B5128216B2B5D5F0F3225F
:10038000D2A3C256D2A2C259C2A1C258D2A4C25745
:10039000C2A0125C2912036FD2A0125C2E12036F4E
:1003A000C2A0125C2912036FD2A0125C2E12036F3E
:1003B000C2A0125C2912036FD2A0125C2E12036F2E
:1003C00012036F12036F12036F12036F22C0F075D6
:1003D000F0DCD5F005B2B512059BC0F012058ED049
:1003E000F030E7EED0F022AAF01203CDE532652F0F
:1003F000F5F0E533653045F0600C1204DD852F32F1
:100400008530331203CD1205531203CD12057B1232
:1004100003CD1204EA8AF022AAF01203CDE5326578
:100420002FF5F0E533653045F0600C1204DD852FC3
:10043000328530331203CD12053F1203CD12057BF6
:100440001203CD1204EA8AF022AAF01203CDE5329B
:10045000652FF5F0E533653045F0600C1204DD855D
:100460002F328530331203CD12050F8AF022AAF005
:100470001203CDE532652FF5F0E533653045F060C8
:100480000C1204DD852F328530331203CD1204F7B0
:100490008AF022C0F075F00833C297928300D29799
:1004A000D5F0F5D0F022C0F075F008C297D29700D1
:1004B000A28233D5F0F5D0F022D2B7D297D283D230
:1004C00082D28422120493E53033E52F3312049351
:1004D000C3E53033120493E531120493221204B9B8
:1004E000C28474531204C4D284221204B9C2847424
:1004F000581204C4D284221204B9C284745412045F
:10050000C4E41204931204A6F608D9F9D284221284
:1005100004B9C28474541204C4E41204931204A6ED
:10052000F208D9F9D284221204B9C2847454120494
:10053000C4E41204931204A6F0A3D9F9D2842212BF
:1005400004B9C28474841204C4E612049308D9F96D
:10055000D284221204B9C28474841204C4E2120444
:100560009308D9F9D284221204B9C2847484120483
:10057000C4E0120493A3D9F9D284221204B9C2842C
:1005800074831204C4D2841281FE1281FE22C284BA
:1005900074571204931204A6D2842275F0641205D3
:1005A0008E20E50430E30122C2AFB2B5128216B24A
:1005B000B5128216D5F0E712038080FBD283D28277
:1005C000D297D2B7D284B2B575F0021281FED5F0BF
:1005D000FAC2B7B2B575F0021281FED5F0FAD2B701
:1005E000B2B5227920752F017530037531E0900086
:1005F000E11203CD1204DD1203CD12052779007537
:100600002F017530047531009001011203CD1204E1
:10061000DD1203CD12052779E0752F0175300575C0
:1006200031009002011203CD1204DD1203CD120538
:1006300027852F3285303322752F017530DB7531D8
:10064000001203CD1208D37532FF7533FF22AE833B
:10065000AD8290DB007F207404F9747FF8752F0160
:1006600085833085823112046E787FE66E702508AE
:10067000E66D702008E6601AB4FF02801316740459
:10068000F9747FF8752F0185833085823112041843
:10069000C322D322A3A3A3A3DFBD80F490DB007FFA
:1006A000207404F9747FF8752F01858330858231B9
:1006B00012046E787FE66E700908E66D700408E635
:1006C000FC22A3A3A3A3DF0A7CFF2290DB007F20F0
:1006D0007BFF7404F9747FF8752F01858330858260
:1006E0003112046E787FE66E702C08E66D70270874
:1006F000ECB4FF0D787F76FF0876FF0876FF08746C
:10070000FFF67404F9747FF8752F018583308582B4
:1007100031120418C322BBFF10787FE6B4FF0A0829
:10072000E6B4FF05C374209FFBA3A3A3A3DFA3BB71
:10073000FF02D322EB232354FC2400F5827583DBD4
:1007400050020583787FEEF608EDF608ECF608E433
:10075000F67404F9747FF8752F0185833085823132
:10076000120418C32275830075F08E752F028583DD
:1007700030753100C0F0C0831203CD1208D3D0838E
:100780000583D0F0D5F0E475830075F0DA752F039A
:10079000858330753100C0F0C0831203CD1208D3B9
:1007A000D0830583D0F0D5F0E47532FF7533FF2296
:1007B00075830075820075F08EC0F0C082C08375AD
:1007C0002F028583307531001203CD1204DDD083F2
:1007D000D082C082C083752F0085823075310012AF
:1007E00003CD12057BD083D08205830582D0F0D55E
:1007F000F0C775830075820075F0DAC0F0C082C062
:1008000083752F038583307531001203CD1204DD0B
:10081000D083D082C082C083752F0185823075312C
:10082000001203CD12057BD083D08205830582D0D0
:10083000F0D5F0C77532FF7533FF227583007582DE
:100840000075F08EC0F0C082C083752F00858330A4
:100850007531001203CD1204DDD083D082C082C076
:1008600083752F028582307531001203CD12057B0E
:10087000D083D08205830582D0F0D5F0C775830080
:1008800075820075F0DAC0F0C082C083752F0185D3
:1008900083307531001203CD1204DDD083D082C0C5
:1008A00082C083752F038582307531001203CD120B
:1008B000057BD083D08205830582D0F0D5F0C77543
:1008C00032FF7533FF221204B9C28474501204C47B
:1008D000D284221204B9C28474811204C4D2842244
:1008E0001204B9C28474841204C4E8120493D9FABD
:1008F000D28422F879001203CD1208E0EAC0E08524
:10090000822F8583307531001203CD12057BD0E034
:10091000FA0583DAE77532FF7533FF221204B9C294
:100920008474541204C4E4120493E4C0E01204A6D4
:10093000D0F025F0D9F5D28422758300758202802B
:1009400006758300758200E475F08D85822F85839E
:1009500030753100C082C083C0F0C0E01203CD12F8
:1009600004DD1203CD790012091CD0F025F0D0F07F
:10097000D083D0820583D5F0D285822F85833075D0
:100980003100C0E01203CD1204DD1203CD79201234
:10099000091CD0F025F07532FF7533FF22758300F6
:1009A0007582038006758300758201E475F0DA852F
:1009B000822F858330753100C082C083C0F0C0E0D3
:1009C0001203CD1204DD1203CD790012091CD0F000
:1009D00025F0D0F0D083D0820583D5F0D27532FFD8
:1009E0007533FF05E02275830075F000752F0085D3
:1009F0008330753100C0F0C0831203CD1208D3D00C
:100A0000830583D0F0D5F0E47532FF7533FF75832D
:100A10000075F0DA752F01858330753100C0F0C0A4
:100A2000831203CD1208D3D0830583D0F0D5F0E430
:100A30007532FF7533FF2253580F53570F5318F079
:100A400053190FC2AFE5572324B0F8E5184519F63E
:100A500008A61A055753570FE557B55805055853BB
:100A6000580FD2AFC3E55795585002241024F450C4
:100A70000375620022E558B557057400780022C35B
:100A80003324B0F8E6C0E008E6F8D0E02253570F70
:100A900053580FC2AFE558B55704D2AFD32205580B
:100AA00053580FD2AFC322300C597884E6540FC08C
:100AB000E0E6C4540375F00AA4D0F025F0FD788573
:100AC000E630E402240A540FFE901A007F3C7404BE
:100AD000F97400F8752F018583308582311204493D
:100AE0007800E26D701708E26E701208E2C42354B9
:100AF000E0F5F07885E6541F45F0F68006A3A3A341
:100B0000A3DFCB2212652C120AA712653BFEAFF0C1
:100B10007DFF0DED30E70122D26575F004A424E1DC
:100B2000F582E5F03400F583C082C083787FE0F67B
:100B3000A308E0F6A308E0F6A308E0F6D083D0828D
:100B4000787F8683088682787FB6FF0708B6FF0322
:100B5000020BCAC3E58233F582E58333F583E58270
:100B600024E0F582E5833405F5837881E6705B083F
:100B7000E66057FB7402F9747FF8752F01858330A6
:100B800085823112046EA3A3787FE60856B4FF0372
:100B9000020BCA787F86F053F07F08E6C39EC5F04B
:100BA0009F401E7025E5F06018BD001E20431B7895
:100BB0007FE6A2E720E713E5F024FA400DD2748027
:100BC00009787FE6A2E79265DBAABD00028028EDE6
:100BD00014C0E0030303540F247AF8D0E054070450
:100BE000FB7400D333DBFD306505FBE24B8004F47E
:100BF000FBE25BF2020B12B2651280DA406E20312A
:100C00006B201B0B204205306562800320655D3040
:100C1000653B20423878B4E2702D20731F78B2E231
:100C2000602B12620A6026F5F07518C0751909E587
:100C3000F0543F4400F51A120A37800512620A6028
:100C40000C78B2E278B4F2D274D273801FC274C24C
:100C500073A2659242400D304312C243120C6F12D0
:100C6000409B8008204305D243120C85020B12C220
:100C70004375186075190F751AE0120A37757E03EF
:100C8000C245C24822D24375187075190F751AE013
:100C9000120A37757E0322120493E53033E52F33B1
:100CA000120493C3E53033D2E0120493E531120409
:100CB00093221204B9C2847454120C97E412049360
:100CC0001204A6F608D9F9D284221204B9C2847497
:100CD00084120C97E612049308D9F9D2842290FC6E
:100CE00000752F04753000753100C082C083754ACD
:100CF000FA1203CD1204DD852F6B85306A790878EE
:100D00007F1203CD120CB2120EDAD083D08270445F
:100D1000C082C08378838683088682120D8B40242C
:100D200078818683088682120D8B4018120DAAE501
:100D300082600AE568B56A0CE569B56B07D083D0B7
:100D400082020D667881E6249AF6120F1D12038046
:100D5000D083D0820530E5307002052FA3E58245AF
:100D6000837087120D6D7532FF7533FF227881769F
:100D7000000876007883760008760008760008760A
:100D800000756B04756A00120EF922C082C083E5FB
:100D9000822400F582E5833480F5834005D083D03A
:100DA0008222D083D08290000022E58275F008A4D0
:100DB000F582E5F0C58375F008A42583F583E5F099
:100DC0003404F569E5822400F582E5833400F58377
:100DD0005002056985836822120380D083D0822265
:100DE000C082C083120EB370EF788186830886823A
:100DF000120D8B40E3120DAA121194787F760078C1
:100E000083E518F608E519F60876000876007408F8
:100E1000F9747FF885692F85833085823112041833
:100E20007404F97483F885692F85833085823112C3
:100E3000046E75F004787F7983E667600280990814
:100E400009D5F0F5120EBA78818683088682A3123E
:100E50000D8B7881A68308A6827883868308868294
:100E6000120D8B7881E66583700A08E6658270044E
:100E7000A3120D8B7883A68308A682C06BC06A85F7
:100E8000696B85686A120EF9D0E0D0F0B56A09C5C1
:100E9000F0B56B028018C5F0C06BC06A85F06BF5C9
:100EA0006A7881E62499F6120F1DD06AD06BD08340
:100EB000D08222120EBA120EDA22856B2F856A308A
:100EC0007531001203CD1204DD7908787F1203CD4D
:100ED000120CB2852F32853033227884E61826181A
:100EE00026182618245566700F7884E6186618664A
:100EF000186618661864996622120F00120F1D22D8
:100F00007884E6182618261826182455F67884E6DC
:100F10001866186618661866186499F622856B2F8D
:100F2000856A307531001203CD1204DD1203CD79CC
:100F300008787F120CCA1203CD12057B1203CD1262
:100F400004EA852F3285303322120EB37030788157
:100F5000E6C0E008E6C0E0088683088682C3D0E0E9
:100F60009582F582D0E09583F58350104582600C20
:100F7000E5822400F582E5833480F583C322900066
:100F800000D322C2B6120F49E433C0E075370074B3
:100F900003124705E51E124705E51F124705745366
:100FA000124705D0E012470574001247057400127D
:100FB0004705E583124705E582124705E5371247E5
:100FC000053099FD22C2B6E5356004F4FF8004FFC8
:100FD000120D6D7537007403124705E51E124705A3
:100FE000E51F1247057456124705EF124705E5370E
:100FF0001247053099FD227401C0E0787F75F00832
:10100000E4F608D5F0FBD0E0D322120F4940E860A7
:10101000E87883868308868212101DC322C082C0AE
:1010200083E58275F008A4F582E5F0C58375F008C4
:10103000A42583F583E5F03404F569E5822400F501
:1010400082E5833400F583500205697408F9747FE2
:10105000F885692F85833085823112046ED083D064
:101060008222120F497F085005120D6D7F00788192
:10107000865908865A08865B08865CC2B6753700B2
:101080007403124705E51E124705E51F1247057454
:1010900054124705E535124705EF124705E535605F
:1010A0003CE55C655AF5F0E55B655945F0600B85FC
:1010B0005C82855B8312101D8003120FF9855C82B0
:1010C000855B83A3120D8B85825C85835B787F753E
:1010D000F008E612470508D5F0F8D535C4E5371213
:1010E00047053099FDC322E5357007C2AF120F499D
:1010F0005005E535F4800C7883A65B08A65C120EDB
:10110000F9E535D2AFC0E0C2B675370074031247B7
:1011100005E51E124705E51F1247057455124705E0
:10112000D0E0124705E5371247053099FDD322C2BA
:10113000B67537007403124705E51E124705E51F13
:1011400012470574581247057420232354FC0412D7
:101150004705742012470590DB007F207404F97462
:101160007FF8752F0185833085823112046E787F78
:10117000E612470508E612470508E612470508E6A5
:1011800012470508A3A3A3A3DFD2E5371247053012
:1011900099FDD32212652C7885E630E402240A54A6
:1011A0000FC4F97884E6C4540375F00AA4F5F0E698
:1011B000540F25F0C313497880F67884E692E754FB
:1011C000C0F97882E6C4540775F00AA4F5F0E65435
:1011D0000F25F049F97883E6C4540375F00AA4F5A5
:1011E000F0E6540F25F0F5F07881E654702345F0D1
:1011F0007882F67881E9F622223044FD125C297566
:10120000F00612011E125C2E75F01412011EE53F4D
:10121000C24422E422787F7910E6B5F0070805F091
:10122000D9F7E422740122C0E0787F7910F608052E
:10123000E0D9FA7410F9747FF8752F037530DB75F7
:1012400031001204187410F9747FF8752F0375308B
:10125000DC7531001204187410F9747FF8752F03CF
:101260007530DB75310012046ED0F0C0F01212152B
:10127000701E7410F9747FF8752F037530DC7531AA
:101280000012046ED0F0C0F01212157003D0F022DC
:10129000D0F022E51DC0E0121227D0F07006E5F074
:1012A000F412122722785574FFF2121407C20C129E
:1012B00009A56001221205E37401F97455F8752F30
:1012C000017530037531A01204497410F9748AF85D
:1012D000752F017530037531C01204497410F9740B
:1012E0009AF8752F017530037531D01204497402D4
:1012F000F97467F8752F017530CE75310012044905
:101300007416F974B5F8752F017530CE7531C012A9
:10131000044978B59000CB75F016E2F008A3D5F03B
:10132000F97416F974B5F8752F017530037531A18C
:101330001204497408F97400F8752F017530D275DC
:10134000310012044978009002F475F008E2F008C8
:10135000A3D5F0F9D20CE422797F77E909E4A22A37
:1013600092E0A22B92E1A22C92E2A20492E3A2428A
:1013700092E4F709A73809A73909A73A7404F97460
:101380007FF8752F0275308E75310012041822D245
:1013900042D243C225C22BA22BB392A5C226C22C95
:1013A000A22CB392A6C202C204A204B392802274F9
:1013B00004F9747FF8752F0275308E7531001204B0
:1013C0006E787FB6E9C908E6A2E0922A9224B39229
:1013D000A7A2E1922B9225B392A5A2E2922C92268B
:1013E000B392A6A2E392029204B39280A2E4924244
:1013F000787F76FF7401F9747FF8752F0275308E4F
:101400007531001204182278B575F016E4F208D58B
:10141000F0FB74FF78BDF278BEF222E8C0E078629B
:10142000E2F570D0E0F822E8C0E07863E2F570D031
:10143000E0F822E8C0E07864E2F570D0E0F82275C8
:10144000F00384B40104741A8017B4020474228077
:1014500010B40304742A8009B40404744280027432
:101460001A227403F9745FF8752F0075308C75318A
:10147000E5120449785FE212143F7862F27860E284
:1014800012143F7863F27861E212143F7864F278C4
:101490005FE224FD9208E224E292097401F9745E8D
:1014A000F8752F0075308C7531E2120449785EE2D0
:1014B00024FD9206E224E29207227403F9745FF895
:1014C000752F0075308C7531E51203E77401F974DE
:1014D0005EF8752F0075308C7531E21203E72279C2
:1014E0007F774809774E0977800977A07404F974EB
:1014F0007FF8752F0075308D753120120418740433
:10150000F9747FF8752F0275308D7531201204182B
:10151000227404F9747FF8752F0075308D753120B1
:1015200012046E7981E7648022E4A22092E0A22175
:1015300092E1A22292E2A20192E3797FF77401F98B
:10154000747FF8752F0075308C7531E812041822FD
:101550007401F9747FF8752F0075308C7531E812BD
:10156000046E797FE7A2E09220A2E19221A2E292AA
:1015700022A2E3920122797FE4A22D92E0A22E9290
:10158000E1A22F92E2A21892E392E492E5A23192B4
:10159000E692E7F709E4A23092E0A23292E1A233A8
:1015A00092E2A23492E3A23692E6A23792E7F709DA
:1015B000E4A23892E0A23A92E2A23B92E3A23C92E9
:1015C000E4A23D92E5A23E92E7F709E577F77404BD
:1015D000F9747FF8752F0075308C7531EC12041892
:1015E000797FE578F4F709E579F4F709E57AF4F716
:1015F0007403F9747FF8752F0075308C7531E9121A
:101600000418227404F9747FF8752F0075308C75F6
:1016100031EC12046E797FE7A2E0922DA2E1922EC6
:10162000A2E2922FA2E39218A2E69231A2E709E782
:10163000A2E09230A2E19232A2E29233A2E392348B
:10164000A2E69236A2E7923709E7A2E09238A2E238
:10165000923AA2E3923BA2E4923CA2E5923DA2E63A
:10166000A2E7923E09E7F5777403F9747FF8752FC6
:101670000075308C7531E912046E797FE7F4F578E6
:1016800009E7F4F57909E7F4F57A22797FF774012F
:10169000F9747FF8752F0075308C7531E4120418D9
:1016A000227401F9747FF8752F0075308C7531E460
:1016B00012046E797FE7227401F9744FF8752F00D8
:1016C00075308C7531FC1203E7227401F9744FF800
:1016D000752F0075308C7531FC12044922784FE269
:1016E00070067850F208F22275F000303C0475F074
:1016F0003CA4AAF075F008A4FBACF0EA75F008A4CD
:101700002CFAC374FD9BFB74FF9A7850F2EB08F23D
:10171000227401F97452F8752F0075308D753100FF
:101720001203E7227401F97452F8752F0075308D99
:10173000753100120449227402F97470F8752F0093
:1017400075308C7531FD1204497402F97472F875A4
:101750002F0075308D753101120449227402F9741D
:1017600070F8752F0075308C7531FD1203E7740227
:10177000F97472F8752F0075308D7531011203E719
:10178000227401F97456F8752F0075308C7531F09C
:101790001203E77401F97457F8752F0075308C75D2
:1017A00031F41203E77401F97458F8752F0075309D
:1017B0008C7531F61203E77401F97459F8752F002E
:1017C00075308C7531F21203E7227401F97456F802
:1017D000752F0075308C7531F01204497401F9745D
:1017E00057F8752F0075308C7531F4120449740167
:1017F000F97458F8752F0075308C7531F61204495C
:101800007401F97459F8752F0075308C7531F21226
:101810000449227401F97438F8752F0075308C75FD
:1018200031F81204187401F97439F8752F00753005
:101830008C7531FA1204187401F9743AF8752F0096
:1018400075308C7531FB120418227401F97438F864
:10185000752F0075308C7531F812046E7401F974AF
:1018600039F8752F0075308C7531FA12046E7401D9
:10187000F9743AF8752F0075308C7531FB12046ECF
:10188000227402F9741EF8752F0075308C7531E0E2
:10189000120418227402F9741EF8752F0075308C2A
:1018A0007531E012046E22E57A54026003756F030D
:1018B00078A07983AA6F80021819E7F5F066540FB3
:1018C000700E18E7C4F5F066540F7004DAEAE422EB
:1018D000E6540FC5F0540FC395F0920B74012278B3
:1018E00084791F7A03E6C4540FF309E6540FF30911
:1018F00008DAF2791F78A37A06E6540FF6E36670E9
:10190000080908DAF4E4C24922792478A87A06C3DF
:10191000E3961918DAFA920B792478A87A06E35438
:101920000FB40F08E6540FB40F108008E6540FB43C
:101930000F0B80061819DAE680CB740122C3E396F8
:10194000B40902801214600FC3E3F5F0E695F0B419
:10195000090280031470E3E9B41F04E4D249221998
:1019600018E366540F60F080D11218DF701D304903
:101970001A20301875185085831985821A120A3773
:101980007548B4757B00D245D248E422042274081D
:10199000F9747FF8752F0075308C7531C012046EA4
:1019A0000218A77408F9747FF8752F0075308C75CC
:1019B00031C012046E121969227405F9747FF8752A
:1019C0002F0075308C7531C0120418227403F9741D
:1019D00084F8752F0075308C7531C512041822C03B
:1019E00082C083E5822420F582E583347DF583740B
:1019F00001F9743BF8752F0085833085823112041C
:101A00006ED083D082C082C083E58275F008A424A2
:101A100020F582500205F0A8F0E58375F008A428AF
:101A20002400F5837408F9747FF8752F00858330DE
:101A300085823112046ED083D082123B5A22C0823A
:101A4000C083E58275F008A42420F582500205F0D9
:101A5000A8F0E58375F008A4282400F5837408F93C
:101A60007497F8752F0085833085823112046ED00B
:101A700083D08222C082C083E58275F008A424202E
:101A8000F582500205F0A8F0E58375F008A428243B
:101A900000F5837406F9747FF8752F00858330850F
:101AA000823112046ED083D082227405F9747FF8DB
:101AB000752F0075300075312012046E0218A79042
:101AC00000001219DF1218A722300CF3751B0075E5
:101AD0001C0075669F75670FE566251BC2E0F582E1
:101AE000E567351CF583C082C083E5822400F5825A
:101AF000E583341BF5837402F9747FF8752F018533
:101B0000833085823112046E787F86830886821244
:101B100019DF1218A77005D0F0D0F022D083D08240
:101B2000C3E58313F583E58213F582200B14E58268
:101B300045836022E58224FFF566E58334FFF5677F
:101B40008007A385821B85831CC3E566951BE5671B
:101B5000951C40028082740122300C397410F97493
:101B60007FF8752F017530CE75312012046E78978D
:101B7000797F75F00AE7B4FF02801AB43C120809B5
:101B8000D5F0F2900FE878C3E2F53B7854F2E42206
:101B900066540F60E97401229000001219DF1219D7
:101BA000692278A3E6540FB40F03021C3C200C02F8
:101BB00080E6751B00751C0075669F75670FE566EE
:101BC000251BC2E0F582E567351CF583C082C08322
:101BD000E5822400F582E583343BF5837402F974D1
:101BE0007FF8752F0185833085823112046E787FEE
:101BF00086830886821219DF1219697005D0F0D029
:101C0000F022D083D082C3E58313F583E58213F5F8
:101C100082200B14E58245836022E58224FFF5666D
:101C2000E58334FFF5678007A385821B85831CC38A
:101C3000E566951BE567951C400280827401227859
:101C4000977A0579ABE6540FC4F5F008E6540F45D2
:101C5000F0F70809DAEF2275F01E1281FED5F0FACE
:101C60001200E475F00F1281FED5F0FA1200E4754F
:101C7000F00F1281FED5F0FA1200E422120094B2A5
:101C8000B575F00F1281FED5F0FA30B7EF22D21AF7
:101C9000D2A3C256C2A2D259D2A1C258D2A4C2570C
:101CA000121C7C121C57121F4112544A1264C81293
:101CB0000D6D120638C2A3C256C2A2C259C2A1C239
:101CC00058D2A4C257125C514005C2AF0261C21281
:101CD0000094B2B575F00F1281FED5F0FA80E6C21D
:101CE000A3C256C2A2C259C2A1C258D2B775F0024D
:101CF0001281FED5F0FA20B744125C515002808E5A
:101D0000D21AD2A3C256C2A2D259D2A1C258D2A4C8
:101D1000C257121C7CD21A125490401CC2A3C25645
:101D2000C2A2C259C2A1C258D2A4C257121E6C127A
:101D3000544A120D6D120638C2AF0261C2125C2EF7
:101D4000C01D120941D0F0703AC3E51D95F0F57C35
:101D5000121E0A1215116019D21A9000001219DF12
:101D6000121E6C12544A120D6D120638B2B5121EB4
:101D70000A1212A5E57A540870081264A5500312DD
:101D80001DC522D2A3C256D2A2C259C2A1C258D2E4
:101D9000A4C257C21A754AFAC2A075F0C81281FED1
:101DA000D5F0FA125C29D2A075F0C81281FED5F0E8
:101DB000FA125C2E1232A7D2B712821620B7C402D2
:101DC0001CF9020000D2B712821630B7F5D2A3C2B6
:101DD00056D2A2C259C2A1C258D2A4C257C21A75C1
:101DE0004AFAC2A075F0141281FED5F0FA125C29ED
:101DF000D2A075F0141281FED5F0FA125C2E1256A4
:101E0000F51232A71264A540BC2212155012160317
:101E10001216A1A2E0923FA2E19240A2E2924112E8
:101E200016CA1217241217CA12184A121737740149
:101E3000F974B2F8752F017530CE7531301204493E
:101E400078B2E2B4FF02E4F27401F974B3F8752FCA
:101E5000017530CE75313112044978B3E2B4FF0216
:101E6000E4F21218941214621216DD22D21AC2A3DE
:101E7000C256C2A2C259C2A1C258D2A4C257C01EE1
:101E8000C01F787F9000007A08E6F008A3DAFA1203
:101E90001F411264C8787F9000007A08E0F608A31A
:101EA000DAFA9000001253B91219B91219CCD01FE6
:101EB000D01E12188122751E30751F30D220C2210B
:101EC000C222C201C22DC22EC22FC218C231C230DC
:101ED000D232C233C234C236C237C238C23AC23B2F
:101EE000C23CC23DC23E75770075780075790075B9
:101EF0007A0878707422F2087400F278727406F22C
:101F0000087400F2C23FC240C241784F7404F278B4
:101F1000527409F278567401F278577402F27858C4
:101F20007404F278597404F2753807753900753AFB
:101F3000007401785EF2785FF2E408F208F2C20CF5
:101F4000221209E6121EB6121881121529121576F0
:101F5000C2E0A23F92E0A24092E1A24192E21216B8
:101F60008B1216B712171112178112181312175C61
:101F70001214BA1214DF125CAB22305B04C25B8015
:101F80000975F00C20B205D5F0FAD322C322E8C0BF
:101F9000E0E9C0E0EAC0E0200637200834121F7AEA
:101FA0005025755000785FE2600C75F0031281FED9
:101FB000D5F0FA1222BC785EE2600C75F003128153
:101FC000FED5F0FA12241DD0E0FAD0E0F9D0E0F806
:101FD0002220092220071F3069EDC082C083E56EF0
:101FE000700812664F400312200D12141B12661F58
:101FF000D083D08280D13069CEC082C083E56E703C
:1020000003122063126728D083D08280BA30050C77
:10201000300609D264C263785E0220253008F4D20B
:1020200063C264785FE2B40F028013B41007123DFC
:1020300009D251802D75F00384E5F0B40007123DFC
:10204000ECD251801DB40107123C77D2508013B4FA
:102050000210123BEE400B784DE583F208E582F268
:10206000D2522230050C300709D264C263785E0276
:10207000207B3009F4D263C264785FE275F0038498
:10208000E5F0B40009123F9F4020D251801CB401FA
:1020900009123FC74014D2508010123FCA400B783B
:1020A0004DE583F208E582F2D25222D2538008C273
:1020B0005312211D753C00C219D25B754AFA744057
:1020C000301A02740CF547C251C244E54760391218
:1020D0001F8E20513375F0031281FED5F0FA1202E3
:1020E0007A201A032019183044E120531B754760E9
:1020F0001211F9B40B0D75F0081281FED5F0FAD269
:1021000051800512211080C3C250D2AF754AFA2205
:10211000533C07F8E53C24A3C8F6053C2278A37598
:10212000F00874FFF608D5F0FB22305009201F0399
:10213000D21F22C25022C21F22D2538004D25BC2BD
:1021400053C219754AFAD21E7440301A02740CF543
:102150004712211D753C00C251C250C244C252C236
:102160005412027A201A0320192D121F8E20512991
:1021700020502620522330442D785EE27004C24461
:1021800080242053147547601211F9B40B1275F0B6
:10219000081281FED5F0FAD251757B03754AFA22F6
:1021A000757B03122110E54760F23054FD80B0B416
:1021B0000207205107C250C25202223DC082C08392
:1021C00090EA60E53C606324FB405F78A3E6540F2F
:1021D000758300F582D53C02805075F00AA4F58223
:1021E00075830008E6540F2582F582D53C02803ABB
:1021F000E58275F00AA4F58285F08308E62582F56C
:102200008250020583D53C028020E58275F00AA445
:10221000F582C0F0E58375F00AA4D0F025F0F583CF
:1022200008E62582F58250020583784DE583F208A1
:10223000E582F2C251C250D252D083D08222C289EA
:10224000C28BD293C2B422C0F075F0FAD5F0FD75FE
:10225000F064D5F0FDD0F02212224712224712225C
:102260004712224712224712224722D293C2B47544
:10227000F00512821620B20612821630B203D5F093
:10228000F112821622C0F075F008A2E7B392B4C230
:1022900093122247C2B4D293122247C0E0E430B274
:1022A00001040030B201040030B20104D36003D550
:1022B000E001C3D0E033D5F0D1D0F022D293C2B444
:1022C000D2B2122247C293122258D293122258201D
:1022D0001A0330641C788F7601087480F608A2A374
:1022E000B392E4F6749008F608F608F608F60223AE
:1022F00031788F7603087680087480A25692E5A222
:10230000A3B392E4201A08A25992E1A22A92E0F61D
:10231000087480201A1220640FE55054074480A2EC
:102320005892E5A2A1B392E4F6087480F608F60884
:10233000F675F007788F7E007F00E62EFEE612220B
:1023400085F62FFF08D5F0F2EED333122285F8EF91
:10235000D333687064788FB6FF5F0560E56024FE54
:102360005014756002201C0ED21C7518C07519001F
:10237000751A03120A37201A08785FE26003306486
:10238000030224197895E620E35920E24920E12749
:102390007890E6B6002108B6420908E6D263122812
:1023A000698076B6551108B6000D08794DE6F30838
:1023B00009E6F3D252D2638060E5606017D56014FD
:1023C000301C11C21C7518C0751900751A04120A48
:1023D00037757D0380437890863C08D25179A37A83
:1023E00004800B7890D250756F0579977A05D26387
:1023F00075F00FE6C4540FF755F0F5F009E6540FE9
:10240000F755F0F5F00908DAEAE5F0B40F051977A9
:10241000EEC250785FE21221AF12226B22D293C239
:10242000B4D2B2122247C293122258D29312225827
:10243000201A1F306323788F7611087480F608A263
:10244000A3B392E4F6749008F608F608F608F602CC
:1024500024A2788F761502245D788F761308768013
:10246000087480A25692E5A2A3B392E4206314A25A
:102470005792E1A2A4B392E0201A08A25992E1A2D5
:102480002A92E0F608748020630FE55054074480D8
:10249000A25892E5A2A1B392E4F6087480F608F679
:1024A00008F675F007788F7E007F00E62EFEE612B4
:1024B0002285F62FFF08D5F0F2EED333122285F8ED
:1024C000EFD333687062788FB6FF5D055FE55F24F8
:1024D000FE5014755F02201D0ED21D7518C07519AF
:1024E00000751A05120A37785EE260033063030252
:1024F00025937895E620E36520E25520E148789021
:10250000E6B6002208B6420A08E6D264122869023A
:102510002593B6551108B6000D08794DE6F3080964
:10252000E6F3D252D264806BE55F6017D55F14305A
:102530001D11C21D7518C0751900751A06120A37CB
:10254000757D03022593D2647890863FD244804300
:102550007890863C08D25179A37A04800B7890D287
:1025600050756F0579977A05D26475F00FE6C454FB
:102570000FF755F0F5F009E6540FF755F0F5F009AF
:1025800008DAEAE5F0B40F051977EEC250785EE29A
:102590001221AF12226B22785FE2601024FD400C02
:1025A00075F0031281FED5F0FA1222BC22785EE2A9
:1025B000601024FD400C75F0031281FED5F0FA1274
:1025C000241D22C0E030630C7518B0751900751A0F
:1025D00000120A37D0E022D293C2B4D2B2122247FC
:1025E000C293122258D293122258788FE573540F57
:1025F000C44407F608E57223A2E392E5A2E292E35F
:10260000542AD2E7F608E572A2E392E1A2E492E34B
:10261000542AD2E7F608E572A2E692E1A2E792E335
:10262000540AD2E7F6748008F608F608F675F00743
:10263000788F7E007F00E62EFEE6122285F62FFFC1
:1026400008D5F0F2EED333122285F8EFD333687059
:102650000B788FB6FF0612226BC3800412226BD355
:10266000227573087874E2F5721225D7740040055C
:10267000122737800312275D7573097875E2F572AA
:102680001225D774014005122737800312275D22D7
:1026900022E577542060F97573047572FF1225D70F
:1026A0007402500412275D2212273778927948E687
:1026B000F30809E6F308794AE6F30809E6F37890A7
:1026C000E6A2E092E25414F5F008E623A2E592E0D7
:1026D000540345F0F5F0784CE265F0C0E0E5F0F227
:1026E000D0E030E21FC0E0C0F0E5F075F04930E224
:1026F0000375F04A7518C075190085F01A120A376B
:10270000D0F0D0E054037003022736E5F05403B450
:10271000030575F0488013B4020575F047800BB4CB
:10272000000575F04B800375F04C7518C0751900E5
:1027300085F01A120A3722F5F02442F8E2B40205B5
:10274000227402F22250FA7402F2E5F02432F5F01B
:102750007518C075190085F01A120A3722F5F02491
:1027600042F8E2601AD5E016F2E5F0243CF5F07587
:1027700018C075190085F01A120A37757D03F22208
:10278000D293C2B4D2B2122247C293122258D29329
:10279000122258788FE573540FC44403F6087680EC
:1027A000087480A25692E5A2A3B392E4A25992E1E2
:1027B000A22A92E0F6087480A25892E5A2A1B392F0
:1027C000E4F6087480F608F608F675F007788F7E50
:1027D000007F00E62EFEE6122285F62FFF08D5F0D8
:1027E000F2EED333122285F8EFD333687071788F0D
:1027F000B6FF6C7895E620E33020E22020E1607897
:1028000090E6B6005A08B6551108B6005208794D40
:10281000E6F30809E6F3D252804A80437890863C7A
:1028200008D25179A37A04800B7890D250756F0545
:1028300079977A0575F00FE6C4540FF755F0F5F067
:1028400009E6540FF755F0F5F00908DAEAE5F0B4B7
:102850000F051977EEC2507865E21221AF8005129C
:10286000226BD32212226BC322B4FF15D270756D76
:10287000051225C37518C0751900751A07120A3795
:1028800022B4BC0302289AB4BD030228CCB4BE0310
:102890000228FEB4BF03022930222063147408F911
:1028A000747FF8752F017530CE75314012046E803B
:1028B000127408F9747FF8752F017530CE753148A0
:1028C00012046E74117887F6122962222063147440
:1028D00008F9747FF8752F017530CE7531501204E8
:1028E0006E80127408F9747FF8752F017530CE75FB
:1028F000315812046E74127887F61229622220630E
:10290000147408F9747FF8752F017530CE75316035
:1029100012046E80127408F9747FF8752F017530F7
:10292000CE75316812046E74137887F6122962220C
:102930002063147408F9747FF8752F017530CE7513
:10294000317012046E80127408F9747FF8752F01CB
:102950007530CE75317812046E74147887F61229AA
:1029600062227880E61201584004741ED3227881D6
:10297000E61201A8400C741FD32212598B1200D703
:10298000C322787FE660F9B4FF08D270756D050246
:102990002B8AB40212203A031225C37887E6126FFD
:1029A000F0400280DB80D3B4090CC0E07404126BE9
:1029B0006DD0E0022B8AB438087882E6122B9B8017
:1029C000BFB439087882E6122BA580B4B43A25301A
:1029D00074201225C378B3E278B4F2788786F07554
:1029E00018C0751909E5F0543F4480F51A120A37EA
:1029F0008088808CB43B223074F81225C3E478B40C
:102A0000F2788786F07518C0751909E5F0543F44CF
:102A100040F51A120A3702297AB43C0D1225C37800
:102A200087861A12712F02297AB43D311225C320EC
:102A30004314D24375187075190F751AE9120A37C5
:102A4000757E0302297AC24375186075190F751ACD
:102A5000E9120A37757E0312409B02297AB43E13AD
:102A6000E5775410600A1225C3E4122BAA02297AD2
:102A7000022980B43F14E5775410600B1225C3740B
:102A8000FF122BAA02297A022980B4400D1225C315
:102A90007887861A12705902297AB4410D1225C31B
:102AA0007887861A12709A02297AB4420D1225C3C9
:102AB0007887861A12708102297AB4430D1225C3D1
:102AC0007887861A12707202297AB4440E74001242
:102AD0006B6D7887E612824A02297AB4450E74003B
:102AE000126B997887E612825902297AB4460974E2
:102AF00000126BB640E880D5B4470E7402126B6DBD
:102B00007887E612826802297AB4480E7402126B42
:102B1000997887E612827702297AB44909740212F9
:102B20006BB640E880D5B44A0E7403126B6D78879B
:102B3000E612828602297AB44B0E7403126B9978DE
:102B400087E612829502297AB44C097403126BB697
:102B500040E880D5B44D181282A47887E6543F44EB
:102B600080F51A75190B7518C0120A3702297AB444
:102B70004E0C3043061225C3022A4602297AB44F6E
:102B8000092043F71225C3022A321225C37518C043
:102B9000751907F51A120A370229801270B878875A
:102BA000E678AFF2221270C280F47874F208F21262
:102BB00026617887E6543F44C0F51A75190B7518DD
:102BC000C0020A37700575621E8002D21522C298B3
:102BD000C29932201AF830991EC299204F057534D7
:102BE000008014C0F0C0E0C0D075D010E534122EC3
:102BF000FED0D0D0E0D0F020980132C298204FFA19
:102C0000C0F0C0E0C0D075D010304E05C24E754047
:102C100000E54424FE4003754402E54020E71FE53B
:102C20004054072324C0C0E07400342DC0E0E5996F
:102C30002205402543F543D0D0D0E0D0F032543FB8
:102C4000232324C1C0E07400342CC0E0E599221590
:102C50006180DE80DCD561FBB54312D213E8C0E0B1
:102C600078AA74FAF2D0E0F875400080CA022DD03C
:102C7000B462FA80BC80BAB42AF380B5F56124C688
:102C8000E56140E924F5E56150E3056180A378182A
:102C9000F21561809C7819F215618095781AF21509
:102CA00061808E781BF215618087781CF215618037
:102CB00080781DF21561022C31781EF21561022C0C
:102CC00031022DE800022C7000022C7500022C77D6
:102CD00000022C7C00022C4F00022C4F00022C4FD3
:102CE00000022C4F00022C8E00022C9500022C9C1E
:102CF00000022CA300022CAA00022CB100022CB965
:102D000000022C5500022C5500022C5500022C55B7
:102D100000022C5500022C5500022C5500022C55A7
:102D200000022C5500022C5500022C5500022C5597
:102D300000022C5500022C5500022C5500022C5587
:102D400000022C5500022C5500022C5500022C5577
:102D500000022C5500022C5500022C5500022C5567
:102D600000022C5500022C5500022C5500022C5557
:102D700000022C5500022C5500022C5500022C5547
:102D800000022C5500022C5500022C5500022C5537
:102D900000022C5500022C5500022C5500022C5527
:102DA00000022C5500022C5500022C5500022C5517
:102DB00000022C5500022C5500022C5500022DE873
:102DC000800E802D803180358038803B8048804661
:102DD000B40909754300754000022C31B4420975ED
:102DE0004300754080022C31754300754000022C71
:102DF00037B51EDC022C31B51FD6022C31F541024D
:102E00002C31F542022C31B543C6754420122E18E0
:102E1000754000022C3780D0854136126019D24FA0
:102E2000E536B44603024785B4470412602F22B446
:102E3000500E854235125FF4C2ACC24F7571072245
:102E4000B45312854235E542700A125FF4C2ACC237
:102E50004F75710222B4540E854235125FF4C2AC34
:102E6000C24F75710122B4550E854235125FF4C20E
:102E7000ACC24F75710322B4560E854235125FF411
:102E8000C2ACC24F75710422B4570E854235125F31
:102E9000F4C2ACC24F75710522B4580E854235128A
:102EA0005FF4C2ACC24F75710622B44E3D85423507
:102EB000E542B4000B125FF4C2ACC24F7571082238
:102EC000B4010B125FF4C2ACC24F75710922B40297
:102ED0000B125FF4C2ACC24F75710E22B4030B1219
:102EE0005FF4C2ACC24F75710F2224BF24E64004C8
:102EF00085423522C24F22C5372537C53722E534F2
:102F000024F0400EE53423241DC0E07400342FC0AB
:102F1000E022759906C24F753400D2B622802F8008
:102F200034803680388039803E80468048805180A9
:102F30004F804D804B80468050800E022FC57534E7
:102F400003F599122EF7053422E535022F737537F4
:102F500000740380ECE51E80E8E51F80E402302960
:102F6000E53775340F80DA120A75122BC488358064
:102F7000D0E53580C9E535A24392E080C1753403C0
:102F8000A8350535E676FF80B8E535C31360321401
:102F9000700BA22792E0B392E1440480D614700B28
:102FA000A22892E0B392E1440880C8147008A229D4
:102FB00092E0440C80BD147008A20392E0440C809F
:102FC000B274FC80AEE5351470257408305C1230A4
:102FD0005D044406809D305E04440380964407806F
:102FE00092A25D92E0A25E92E1A22A92E280841413
:102FF00070157410A22792E0A22892E1A22992E211
:10300000A20392E3022F7314700D7418A21C92E0B5
:10301000A21D92E1022F7314700BA25F92E0A261D5
:1030200092E2022F73E4022F73E536B44106753441
:1030300004022F41B44212E5356003301503120A31
:103040008D75621E7442022F3EB4440280F8B44B68
:103050000280030230EEE53554F8B4083EE53554FD
:1030600007700B751A19127059E536023123B40135
:103070000B751A19127072E536023123B4020B7502
:103080001A19127081E536023123B4030B751A192F
:1030900012709AE536023123022F12B42003022F58
:1030A00012B42826E53520E00830430B12409B80FF
:1030B00006204303126245E535A2E09243756C0198
:1030C0005003756C02E536022F3EB4300CE53554E2
:1030D000F8126B6DE536022F3EB4380CE53554F826
:1030E000126B99E536022F3E022F12022F12B443C3
:1030F0000FB535037545037534077535AB022F41A0
:10310000B44A26E535701F205E1C205C0874191235
:103110005C33125C2175181075190F751AF0120ABC
:1031200037E536022F3E022F12B4450675340602EB
:103130002F41B4510675340C022F41B44D0EE535C4
:10314000126E7BE5365002B2E7023046B44C06758B
:10315000340E022F41B4460280C9B4470280C4B481
:103160004F08C245C246C24780B9B4590FE5357011
:103170000B857C35745975340D022F41022F12E5F1
:1031800071B4000122B40717C2AC12822E12822E33
:10319000D2991232B8C24FD2B6125FF40232A3B43F
:1031A0000117C2AC12822E12822ED299121062C264
:1031B0004FD2B6125FF40232A3B40317C2AC12822C
:1031C0002E12822ED2991210E7C24FD2B6125FF49D
:1031D0000232A3B40217C2AC12822E12822ED299EE
:1031E000120F83C24FD2B6125FF40232A3B4041797
:1031F000C2AC12822E12822ED299120FC5C24FD2A9
:10320000B6125FF40232A3B40517C2AC12822E12BA
:10321000822ED2991202D4C24FD2B6125FF4023279
:10322000A3B40617C2AC12822E12822ED2991211AA
:103230002FC24FD2B6125FF40232A3B40817C2AC49
:1032400012822E12822ED299125ACBC24FD2B612AD
:103250005FF40232A3B40917C2AC12822E12822E7E
:10326000D299125A4FC24FD2B6125FF40232A3B4AF
:103270000E17C2AC12822E12822ED299125B58C245
:103280004FD2B6125FF40232A3B40F17C2AC12824F
:103290002E12822ED299125B9AC24FD2B6125FF4CE
:1032A0000232A375710022E571B4000122C24FD22F
:1032B000B6125FF475710022125DEBC2B67537006D
:1032C0007403124705E51E124705E51F12470574F2
:1032D00050124705747D124705900000E535600FD8
:1032E0009003E81460099007D0146003900BB87E37
:1032F0007D7F0875F000C0F0125DEBB40203D3804F
:1033000001C3D0E033F5F0A3DFEC124705DEE2E5C0
:10331000371247053099FD22E563C2676002D26724
:10332000E551F552C24820520C20501B3051030287
:10333000344D02391D120102784DE2F58308E2F5A1
:10334000821219DF02350A120102121C3F121AC939
:103350006017121B59603C1225C375182075190F90
:10336000751AEC120A37023396206305205F0A8033
:10337000032061051239C9501AC082C0831200E4CB
:103380001220AFD083D08230510CE53C6008121976
:1033900069700302350A75493CD545177518C07523
:1033A0001900751A53120A37754503757B00D2460A
:1033B0007548B402390AD270756D051225C37518A7
:1033C000C0751900751A07120A377550041225972F
:1033D0001225AD75F06412011E02391D206324E52B
:1033E00079540860CE300C18C0E0C082C0837411DC
:1033F000120188D083D082D0E0400280B902342408
:10340000023424E578548060AA300C18C0E0C082F1
:10341000C0837410120188D083D082D0E040028033
:1034200095023424127173401E205E15302E032045
:103430004309900FE912392602391D1238A20239C8
:103440001D1238A802391D1238AE02391D120102B0
:10345000E53C608878A3E6B40A0302408D121BA203
:10346000707D206305205F50800320614B1239C9B5
:103470004046206325300C19C0E0C082C08374131D
:10348000120188D083D082D0E0400302350A023492
:103490009402350A12387E023396300C18C0E0C010
:1034A00082C0837412120188D083D082D0E040039E
:1034B00002350A80DF02350A1200E4C082C083129E
:1034C000213DD083D082305013C082C083120102CC
:1034D000121C3FD083D0821218A7602E0233967838
:1034E0005E206402785FE2B40F0A123CC1C251D27E
:1034F0005002334AB4100280F11225C375182075AA
:10350000190F751AEB120A3780D2306330300C195C
:10351000C0E0C082C083740C120188D083D082D0F6
:10352000E0400302353D0235297573027860E27888
:1035300065F2121427123E3A50030233963064307B
:10354000300C19C0E0C082C083740D120188D08392
:10355000D082D0E0400302357002355C7573037889
:1035600061E27865F2121433123E3A500302339648
:103570001261EF400312223EE53B047003023396D2
:10358000754900754503C247C246204802C245C07E
:1035900082C083123A70D083D08250061238BD02A6
:1035A000391DC082C08312064ED083D082500612CD
:1035B00038BD02391DE58224CEE58334FF50171251
:1035C00039B74012C216C2171280DA50061238AE4E
:1035D00002391D0237B612717350121238AE02371B
:1035E0005A1238A802375A1238A202375A205EF10E
:1035F000302E032043F13063037854E2306402E557
:103600003B120158500902365312389C02375A3087
:103610000CF73018F4303DF1123F914036A2633080
:103620003E01B3502E300C18C0E0C082C083740934
:10363000120188D083D082D0E0400280CC02364094
:10364000C082C083125E3FD083D08250061238B34E
:1036500002375A301825D239300C19C0E0C082C068
:10366000837414120188D083D082D0E040030236E4
:1036700076023674C239123F9150030236EB125D66
:10368000EBA2E09216A2E19217A263303E01B3C012
:10369000E0920A501E125E95501930390EE4A216BF
:1036A00092E0A21792E1B402028008D0E012388AB8
:1036B00002375AD0E0B40005200A22802BB4012240
:1036C000200A1A7518C0751900751A09120A3720D0
:1036D00039061238B802375A12397A800E125D3E16
:1036E0008009B402ED200ADB125D96300C58123FBF
:1036F000914053300C19C0E0C082C083740812019D
:1037000088D083D082D0E0400302374602370F20B2
:10371000671AA2639266858364858265123976C2D0
:1037200063C2641200F875630202391D756300E517
:10373000836564F5F0E582656545F070061238C270
:1037400002375A12402E123926E5775410600BC00A
:1037500082C083123B80D083D0821239C0500912BC
:103760003B5A30E10302391D1280DA40F8C2A1D27F
:1037700058D2A4C2577550001225971225AD1219C0
:10378000DFC082C08312213DD083D0822052092025
:10379000501720511C02391D120102784DE2B583E9
:1037A0000D08E2B582080237B61218A76008023980
:1037B0000A12196970F8301824E4A21692E0A217D0
:1037C00092E1B40305125DC28013B40205125D3E9E
:1037D000800BB40105125D968003125D15300C1943
:1037E000C0E0C082C0837406120188D083D082D02A
:1037F000E0400302390A0237F9E5775401601FE51A
:1038000082458360193063037854E2306402E53BFB
:10381000120158500302381E12389002391D1271DD
:1038200086500F12389675F01E12011E1200C1024A
:10383000391DB2431225C330432075187085831992
:1038400085821A120A37757E03C2A3C256D2A1C25C
:1038500058D2A4C257126245801E7518608583191C
:1038600085821A120A37757E03D2A3C256D2A1C22C
:1038700058C2A4C25712409B1200D702391D1259D8
:10388000810238C51259810238C51259810238C5E2
:103890001259810238C51259810238C51259810264
:1038A00038C51259810238C51259810238C51259DA
:1038B000818012125981800D12598180081259811C
:1038C00080031259817563007564FF7565FFD277B7
:1038D0001225C375182085831985821A120A37129A
:1038E00000C1C27722E5785408700320631BE551BC
:1038F00004601614F5F07855E265F0600C7518C098
:1039000075190185511A120A3722125981D277127C
:1039100000ABC2777563007564FF7565FFC251C265
:1039200050E552F5512230430EC2A3C256C2A2C284
:1039300059D2A4C257800CD2A3C256C2A2C259C245
:10394000A4C257A263920ED20D125981741C125C4C
:1039500033125C21E5775440600620A803128101F0
:103960001225C31238E575181085831985821A123D
:103970000A371200D7221259812212598175F0326A
:1039800012011E227408F9747FF8752F0175300337
:1039900075319012046E7884E60856085604601457
:1039A0001200E41220AF305109E53C60051219699C
:1039B0006002C322D32222E582249CE58334FF22C5
:1039C000E582249CE58334FF22A240E582458360A2
:1039D00010E582249CE58334FF5004A23F8002A2BC
:1039E0004122E5822582F582E5833583F583E582F0
:1039F0002582F582E5833583F583E5822400F5820F
:103A0000E583345BF5837404F97400F8752F018540
:103A10008330858231120449227884E654C0F583CC
:103A20007885E630E402240A2323543C4583F58359
:103A30007884E6C4540375F00AA4F5F0E6540F2523
:103A4000F0030303F5F053F0E085F082540345835F
:103A5000F5837883E6C4540375F00AA4F5F0E654C0
:103A60000F25F04582F58222C39582E5F0958322E9
:103A7000123F915003023AF81239E27800E2B4FFA3
:103A800003023AF812652C123A19787FA68308A629
:103A9000827800E2F58308E2F58208E2F5F008E2B8
:103AA000123A68502B7800E2F58308E2F582787FBD
:103AB00086F008E6123A6850417802E2F58308E29F
:103AC000F582787F86F008E6123A68402D023AF8CF
:103AD0007800E2F58308E2F582787F86F008E61246
:103AE0003A6840167802E2F58308E2F582787F862C
:103AF000F008E6123A685002C322D322C3E58233AB
:103B0000F582E58333F583E5822400F582E583348D
:103B10009AF5837402F97453F8752F018583308503
:103B2000823112044922C3E58233F582E58333F5FD
:103B300083E5822400F582E583349AF5837402F9E3
:103B40007453F8752F018583308582311203E72283
:103B500078537400F208E4F2801E300CF3C082C087
:103B600083123AFCD083D082E5822418E58334FCAA
:103B700040067853E24402F27854E2F5F018E2226B
:103B8000E5822400F582E58334BAF5837401F97483
:103B90007FF8752F0185833085823112046E787F1E
:103BA000E660422323C0E05403F5F0D0E054FC2447
:103BB00000F582E5F034CAF5837404F9747FF87572
:103BC0002F0185833085823112046E787FE6088666
:103BD000F07874F208E5F0F275F0021281FED5F08B
:103BE000FA1226612274FF7874F208F280EAE57016
:103BF000B4220575F0048013B42A0575F006800B15
:103C0000B4420575F00C800375F002782EE2540F73
:103C1000704F08D5F0F7E2540F75F00AA4F58275DD
:103C2000830008E2540F2582F582E58275F00AA42C
:103C3000F58285F08308E22582F58250020583E54E
:103C40008275F00AA4F582C0F0E58375F00AA4D06D
:103C5000F025F0F58308E22582F58250020583C342
:103C600022D322782EE2600BF5F008E2240A400508
:103C7000D5F0F7C322D322782E7997770009770001
:103C8000097700097700E570B4220A756F04799905
:103C900075F0088024B42A0A756F05799775F00AC3
:103CA0008017B4420C756F05799775F00A783480E7
:103CB00008756F03799B75F006E2F70809D5F0F9EE
:103CC00022C082C08378979002E175F00AE0F6087E
:103CD000A3D5F0F99002EBE0F56FD083D08222C03B
:103CE00082C08378979002E175F00AE6F008A3D5C8
:103CF000F0F9E56F9002EBF0D083D08222123C778E
:103D00001218A722D083D08222123C77123CDF12F5
:103D1000211DC082C083753C01782EE2540F70E4EF
:103D200008E2540F70DE08E2540FC4F5F008E254C4
:103D30000F45F0F58308E2540FC4F5F008E2540F84
:103D400045F0F582C26D78A37900C3E5829410F541
:103D500082E5839427F58340030980EEE5822410F1
:103D6000F582E5833427F583E96004D26DF608799E
:103D700000C3E58294E8F582E5839403F58340036C
:103D80000980EEE58224E8F582E5833403F583E9D2
:103D9000206D046004D26DF6087900C3E582946456
:103DA000F582E5839400F58340030980EEE58224E3
:103DB00064F582E5833400F583E9206D046004D264
:103DC0006DF608E58275F00A84206D026002F6083F
:103DD000E5F0F6E8245EF53CD083D0822279A37723
:103DE000000975F00577FF09D5F0FA22123C771229
:103DF0003CDF123DDD75F008E570B42204782E80BA
:103E000013B42A047830800CB442047836800578E4
:103E10002E75F006753C06E2540F700608D5F0F7D3
:103E2000800979A3E2F70809D5F0F922123DEC12D6
:103E3000196922123D09121969227865E27003029C
:103E40003EEF24FD4038C082C0831200E4123F4B95
:103E5000D083D08220521620510B3050361218A732
:103E60007031023EEF1219697029023EEF784DE27F
:103E7000B5832008E2B5821B658270178071E22449
:103E8000E24070C082C0831200E41266F1D083D099
:103E9000825003023EF17865E2B40F0C123E2C60B2
:103EA0004E123CFD604980EBB41007123E33603F78
:103EB00080E175F00384E5F0B40007123E2C70D366
:103EC000802DB40107123CFD70C98023B4021EC0CE
:103ED00082C083123BEEE5828583F0D083D082409E
:103EE000B2658270AEE5F0658370A8800280A4C3DD
:103EF00022D322C082C0831200E4126747D083D04D
:103F0000825002D3227865E275F00384E5F0B400B4
:103F10000A123F9F12196970EA802CB4010A123FFD
:103F2000C71218A770DD801FB4021EC082C08312A2
:103F30003FCAE5828583F0D083D08240C665827017
:103F4000C2E5F0658370BCC32280B8754732D25B8E
:103F5000305409C254C07312027AD073E547D3605B
:103F600018C252C251C250121F7A50E41227802048
:103F700052062051033050D8C3C0D0A8737405B87E
:103F800002027404D0D04005122737800312275D47
:103F900022E582B4E807E583B40F02D322C32212DC
:103FA0003C635002D322782EE260F9F5F008753CAC
:103FB00006E2540F700608D5F0F7800979A3E2F7FE
:103FC0000809D5F0F9C322026869123C635004D392
:103FD00022C322782EE20860F6B40108E2F5827569
:103FE000830080EDB40212E275F00AA4F58208E2C3
:103FF0002582F58275830080D8B40320E275F00A2B
:10400000A4F58208E2258275F00AA4F58285F08382
:1040100008E22582F58250B9058380B5B40405789D
:104020002F023C16C39404F5F0782F023C0DB263C6
:10403000B2647550071225971225ADB264B263754C
:1040400018C0751900751A0C120A3730660C7518ED
:10405000B0751900751A00120A371238E575181074
:1040600085641985651A120A3722E53CB4031C7869
:10407000A3E6B40A1608E624F6401008E624F64043
:104080000A18E675F00AA40826C322D32212406A51
:10409000500302345D78ADF20240EA1262451282AA
:1040A000A4C245C2482241414163419F41CB41E204
:1040B00041F9421042274236424542544263429AF5
:1040C00042C542CD42DF42EE432A437C439F43B682
:1040D00043D743F3440F441B44374453445F447B6A
:1040E000449744A344BC4115411578ADE224E04017
:1040F00024124605401378ADE225E0049040A693D3
:10410000C0E0E225E093C0E0220246BD1246BC12A8
:1041100000D702391D740A0246BDD2A1C258C2A4FA
:10412000D2571246BB1200E412213D205102D32285
:10413000E53CB402F978A3E624F640F208E624F65A
:10414000221246BA12411A401578A3E62430F51E11
:1041500008E62430F51F12188112544A80AE7420EC
:104160000246BD1246BA1245A4402F12652C78A310
:10417000E6C40846F5F078A7E65403030345F07853
:1041800084F678A5E6C40846F5F078A8E6C4234589
:10419000F07885F61264DE02410C741E0246BD12F0
:1041A00046BA124555401F12652C78A3E6C408464E
:1041B0007883F678A5E6C408467882F6E47881F636
:1041C0001264DE02410C741F0246BD1246BA12464A
:1041D0009E7518C0751900751A0F120A37D25F0242
:1041E000410C1246BA12469E7518C0751900751A10
:1041F00010120A37C25F02410C1246BA12469E756F
:1042000018C0751900751A51120A37D26102410C93
:104210001246BA12469E7518C0751900751A5212C8
:104220000A37C26102410C1246BA12469E751A1B29
:1042300012705902410C1246BA12469E751A1B1290
:10424000707202410C1246BA12469E751A1B127009
:104250009A02410C1246BA12469E751A1B127081C0
:1042600002410C1246BA1280DA402A12469E1262AD
:10427000451282A4C245C248C243784DE2F5830884
:10428000E2F58275186085831985821A120A3775DE
:104290007E0302410C74160246BD1246BA1280DA41
:1042A00040F312469E126245D243784DE2F58308F0
:1042B000E2F58275187085831985821A120A37759E
:1042C0007E0302410C1246BA20439880CD1246BAB2
:1042D00012469E75F0C81281FED5F0FA0261C21234
:1042E00046BA12469E751A1B12712F02410C1246D5
:1042F000BA20190D12451D402C1246D0402778AE29
:10430000F278AEE2F551F55212469E7518C085510D
:104310001A751903301903751902120A3702410C74
:1043200074190246BD741A0246BD1246BA20190D10
:1043300012451D40F01246D040EB78AEF278AEE266
:10434000F55112469E7518C085511A751906301917
:1043500003751905120A371256F512572C1239B681
:10436000D2A2C259C2A1D2581200E412213D74183F
:104370002050062051033052AE0233261246BA3086
:10438000742D78B3E278B4F212469E7518C0751990
:1043900009741B543F4480F51A120A3702410C126B
:1043A00046BA30740A12451D500A741C0246BD7488
:1043B0001D0246BD70CF1246BA3074F3E478B4F2F1
:1043C00012469E7518C0751909741B543F4440F578
:1043D0001A120A3702410C1246BA7400126B6D753C
:1043E00018C075190A741B543F4400F51A120A3795
:1043F00002410C1246BA7400126B997518C07519F7
:104400000A741B543F4480F51A120A3702410C12F9
:1044100046BA7400126BB640DD80BF1246BA740211
:10442000126B6D7518C075190C741B543F4400F560
:104430001A120A3702410C1246BA7402126B9975AD
:1044400018C075190C741B543F4440F51A120A37F2
:1044500002410C1246BA7402126BB640DD80BF12E4
:1044600046BA7403126B6D7518C075190C741B5421
:104470003F4480F51A120A3702410C1246BA7403FF
:10448000126B997518C075190C741B543F44C0F514
:104490001A120A3702410C1246BA7403126BB64064
:1044A000DD80BF7404126B6D7518C075190B741B19
:1044B000543F4440F51A120A3702410C1282A47587
:1044C00018C075190B741B543F4480F51A120A3733
:1044D00002410CC2A1D258C2A4D2571239B612005E
:1044E000E412213D20520820501C205129D322786B
:1044F0004DE2F58308E2F582120102300C06123B10
:104500005A20E2E9C322121AC970E2784DE583F21B
:1045100008E582F280E2121BA270D280EED2A1C224
:1045200058C2A4D2571246BB1200E412213D2051BA
:1045300002D322E53C60FA24FC40F6A93C78A37A39
:1045400000EA75F00AA42640E8C5F070E4AAF00875
:10455000D9EFEAC322D2A1C258C2A4D2571246BB95
:104560001200E412213D205102D322E53CB404F9AB
:10457000F5F078A3E624F640F008D5F0F778A3E646
:1045800075F00AA4082624E8402E78A5E675F00AFE
:10459000A4082624C4402122E0E2E0E1E0E1E0E0DA
:1045A000E1E0E1E0D2A1C258C2A4D2571246BB1248
:1045B00000E412213D205102D322E53CB406F9F576
:1045C000F078A3E624F640F008D5F0F778A5E67574
:1045D000F00AA4082660E1C0E024F3D0E040D990BE
:1045E000459793F978A3E675F00AA4082660C9C038
:1045F000E029D0E040C278A7E624F640BB78A8E6E0
:1046000024F940B422300C7C784D740FF20874E920
:10461000F220197C78ADE22400F5827583D0740114
:10462000F9747FF8752F0185833085823112046E0D
:10463000787FE6120158506278ADE22400F5827569
:1046400083D17401F9747FF8752F018583308582D9
:104650003112046E787FE61201A8503678ADE2245C
:1046600000F5827583CF7401F9747FF8752F018589
:10467000833085823112046E787FE620630C20E05F
:104680001530E10C1244D3740D2220E20920E3F42A
:10469000C322740E8006740C8002740BD32220197E
:1046A000181225C3784DE2F58308E2F5827518E00B
:1046B00085831985821A120A3722222222C0E0122B
:1046C00059811246BAD0E012556E1200AB02391D64
:1046D000C051C082C083F5511255F1D083D082E51C
:1046E00051D051B322C5372537C53722E54924E9D2
:1046F0004008D2A3C256D2A2C2593098EFC298E560
:10470000991246E5223099FDC299F5991246E522A3
:10471000C2A3C256C2A2C259C2B6753700740512EE
:104720004705E51E124705E51F1247052212822E96
:1047300012822E12822E124710E536124705E537F7
:104740001247053099FD221209A50247501209416E
:10475000C0E0124710E536124705D0E0124705E5E4
:10476000371247053099FD2212822E124710E53686
:10477000124705797FE712470509DDF9E53712474A
:10478000053099FD22D21A754919751A001282A4B2
:10479000E538600B54F87007C22BA22BB392A5E545
:1047A00039600B54F87007C22CA22CB392A6E53ADC
:1047B000600B54F87007C204A204B39280125C2EFE
:1047C000C28EC28CC2ADC2ABC2ACC2AF7581D49036
:1047D00047DAC082C08375D00032D2AFD28C125F6C
:1047E000F4C2ACD29912472DB2B5754919D29802CC
:1047F0004817B40922F5371246ECB51E271246ECCD
:10480000B51F211246ECB4461B1246ECAF371246D8
:10481000EC6F701012472DD2B6D2A3C256D2A2C2EC
:10482000591246ECB40ACBF5371246ECB51EF51218
:1048300046ECB51FEF1246ECF536B46D030248C7DF
:10484000B46E030248E0B46F03024917B470030268
:104850004964B47103024978B47303024989B4749A
:104860000302498BB4750302499FB47603024914CD
:10487000B477030249B7B478030249CBB479030291
:1048800049ECB47A03024A08B46C03024A1CB46BC4
:1048900003024A3EB46A03024A79B46903024A95A4
:1048A000B46803024AF4B46703024B0CB466030213
:1048B0004B27B46503024BEBB463030252F6B461B9
:1048C00003025361024817AF371246EC6F70F512BE
:1048D000472DD2B675F01E1281FED5F0FA0261C2E4
:1048E0001246ECFD1424E0402B1246EC2400FC7B25
:1048F000001246ECFEAF371246EC6F70178EF0EDEB
:10490000F9747FF88B2F8C3085F03112046E1247CA
:10491000687549190248171246ECFD1454E070F40A
:104920001246EC2400FC247140EA7B021246ECFEA5
:10493000EDFA787F1246ECF608DAF9AF371246EC5A
:104940006F70D1C2A3C256C2A2C2598EF0EDF974E3
:104950007FF88B2F8C3085F0311204181247367592
:10496000491980B0AF371246EC6F70A81207651274
:10497000472D754919024817AF371246EC6F700979
:1049800012474D75491902481780891246ECFD14EB
:1049900024E040341246EC2400FC7B010248F11272
:1049A00046ECFD1454E070201246EC2400FC242553
:1049B00040167B0302492CAF371246EC6F70091288
:1049C000474775491902481702491479187D07129B
:1049D00046ECF309DDFCAF371246EC6F70EA125576
:1049E0007040E51264DE124736024817AF371246B0
:1049F000EC6F70D412652C12822E124710E536121D
:104A000047051202F0024817AF371246EC6F706686
:104A1000120D6D12472D7549190248171246ECFE0A
:104A20001246ECFD1246ECFCAF371246EC6F7046B6
:104A30001206CB404112472D7549190248171246FC
:104A4000ECFE1246ECFDAF371246EC6F70281206F2
:104A50009C12822E12822E124710E536124705EE66
:104A6000124705ED124705EC124705E537124705D9
:104A70003099FD024817024914AF371246EC6F70A7
:104A8000F512822E12822E124710E53612470512B9
:104A90001148024817AF371246EC6F70D912093926
:104AA00060027401C0E012099D60027402D0F045FA
:104AB000F0700A1207B01214DF120D6DE4C0E0129C
:104AC0004710E536124705D0E0C0E0124705E5374C
:104AD00012470575F0031281FED5F0FA124710E572
:104AE00036124705D0E0124705E5371247053099E1
:104AF000FD0248171246ECFD1454E070271246ECF4
:104B00002400FC2471401D7B0002492C1246ECFD60
:104B10001454E0700F1246EC2400FC242540057B61
:104B20000102492C024914AF371246EC6F70F5129E
:104B3000822E12822E124710E53612470574021299
:104B40004705744E12470574801247057448124792
:104B50000574341247057400124705748D12470519
:104B6000742012470574DA12470574001247057461
:104B70000F12470574A01247057480124705740090
:104B8000124705740012470574201247057400127D
:104B90004705740012470574001247057400124758
:104BA000057400124705740012470574001247058A
:104BB000740012470574001247057400124705740B
:104BC000001247057400124705740012470574006F
:104BD00012470574001247057400124705E53712A5
:104BE00047053099FD0248170249141246ECF58337
:104BF0001246ECF5822460E58334F040EB124E77E8
:104C00001246ECFD1454E070DF780075F02074FF5C
:104C1000F208D5F0FB78001246ECF208DDF9AF3768
:104C20001246EC6F70C212472D75F0051281FED549
:104C3000F0FA124736751A01300CAD124EAD124E15
:104C400093124E851219DF789779007A0A75F00F62
:104C5000E3540FF652F00809DAF643F0F0E5F004F9
:104C600078A079837A051218BA600B124D0C5006A1
:104C7000751A04024BE8124E93124E851219DF7812
:104C8000A3790A7A0675F00FE3540FF652F008097B
:104C9000DAF643F0F0E5F00478A879867A03121882
:104CA000BA600B124DAA5006751A06024BE8124E56
:104CB00093124EF6751A65024817C0E07828E5830E
:104CC000F208E582F2D0E022C0E0782AE583F2081B
:104CD000E582F2D0E022C0E07828E2F58308E2F530
:104CE00082D0E022C0E0782AE2F58308E2F582D0A3
:104CF000E022E5822400F582E583341BF58322E57A
:104D0000822400F582E583343BF58322124E85AB85
:104D100083AC82901B00C0837900752F038583309C
:104D20007531009000561203CD1204DD1203CD122E
:104D300005279000567A80E0A3F5F0E0A36C70059B
:104D4000E5F06B6017DAF0D0830583740024C0E5CA
:104D50008334C550C17405124E59D322D083EA2A38
:104D6000F5F0E4C395F0F582124CBA789779007AA1
:104D70000A75F00FE3540FF652F00809DAF643F023
:104D8000F0E5F004600C121ACC700A7406124E5949
:104D9000D322121ACCE5822582F582E5833583F58C
:104DA00083124CF2124CC80250FE124E85AB83ACFB
:104DB00082903B00C0837900752F03858330753165
:104DC000009000561203CD1204DD1203CD12052708
:104DD0009000567A80E0A3F5F0E0A36C7005E5F052
:104DE0006B6017DAF0D0830583740024C0E5833448
:104DF000A550C17405124E59D322D083EA2AF5F08A
:104E0000E4C395F0F582124CBA78A3790A7A067554
:104E1000F00FE3540FF652F00809DAF643F0F0E52C
:104E2000F004601D121BB2701BAB83AC82124E8566
:104E3000EBB58306ECB58202C3227404124E59D33B
:104E400022121BB2E5822582F582E5833583F58344
:104E5000124CFF124CC80250FEF51A22C082C083C9
:104E6000E58312556FD083D082C082C083E5821261
:104E7000556FD083D08222C0E0782CE583F208E51C
:104E800082F2D0E022C0E0782CE2F58308E2F582DD
:104E9000D0E0227400124705740012470574001216
:104EA0004705740012470574001247052275831BDD
:104EB00075821B75F040C0F0C082C083752F0185DC
:104EC00083307531001203CD1204DDD083D082C04F
:104ED00082C083752F038582307531001203CD1295
:104EE000057BD083D08205830582D0F0D5F0C775CD
:104EF00032FF7533FF227401F97418F8752F0075AD
:104F0000300075310012046E7401F97419F8752FB0
:104F1000017530D97531FF12046EAC18124E85E55B
:104F2000822420F582E583347DF583C082C08374BA
:104F300001F9743BF8752F008583308582311204A6
:104F40006ED083D0827401F97410F8752F008583B8
:104F5000308582311203E77810E2F5F0E518253B41
:104F6000C395F0F518124E85123AFC7853797FE21A
:104F7000F72519F5190809E2F72519F519781679B1
:104F800053E2F3FA0809E2F32AFAC3E5199AF5198C
:104F9000124E85123B26124E85E58275F008A42438
:104FA00020F582500205F0A8F0E58375F008A428EA
:104FB0002400F5837408F9747FF8752F0085833019
:104FC00085823112046E787FE5187A082608DAFCAB
:104FD000F518789779007A0A75F00FE3540FF652B6
:104FE000F00809DAF643F0F0E5F00412550C78A366
:104FF000790A7A0675F00FE3540FF652F00809DAD1
:10500000F643F0F0E5F0041255147408F9747FF8D3
:10501000752F00858330858231120418787FE5185A
:105020007A08C39608DAFBF518124E85C3E5823379
:10503000F582E58333F583C3E58233F582E5833377
:10504000F583E5822400F582E583245BF583C08245
:10505000C0837404F9747FF8752F018583308582CD
:105060003112046ED083D0827404F97412F8752F53
:10507000018583308582311203E7787F7912E51943
:105080007A0426F5F0E3C5F0C395F00809DAF3F5E4
:10509000197401F97418F8752F0075300075310016
:1050A0001204187401F97419F8752F017530D97547
:1050B00031FF12041875831B75821B75F040C0F018
:1050C000C082C083752F038583307531001203CDF4
:1050D0001204DDD083D082C082C083752F01858207
:1050E000307531001203CD12057BD083D082058349
:1050F0000582D0F0D5F0C77532FF7533FF22124C10
:10510000E4E5828583F0124CD6C39582C0E0E5F0D9
:105110009583D0F045F07002C32250030252191259
:105120004CE4C0E0C3E58224FEF582E58334FFF55C
:1051300083D0E0124CC8E5828583F0124CD6B5824C
:1051400007E5F0B58302C322124CD6AF83124CE4BC
:10515000EFB58310AE8290002C787FE0F6A308E0D4
:10516000F602517C7EFE8F8305837402F9747FF80A
:10517000752F0385833075310012046E7900752F09
:10518000038F307531009000561203CD1204DD12EA
:1051900003CD1205278F83758200124CD67D00E562
:1051A000836F7002AD82ED2456F582758300500244
:1051B0000583C3EE9D20E05A03FCC082C083A3A3F5
:1051C000E0FAA3E0FBD083D082EAF0A3EBF0A3DC0B
:1051D000E9EE2456F58275830050020583787FE658
:1051E000F0A308E6F07900752F038F307531009039
:1051F00000561203CD1205671203CD12057B852FD1
:1052000032853033124CE4EFB583030252ED0F02C6
:10521000514D7408124E59D322124CD6AF83124C02
:10522000E4EFB58310AE8290002C787FE0F6A308FF
:10523000E0F602524D7E008F8315837402F9747F6D
:10524000F8752F038583307531FE12046E79007571
:105250002F038F307531009000561203CD1204DDFC
:105260001203CD120527124CD67DFEE5836F700226
:10527000AD82ED2456F58275830050020583C3ED9F
:105280009E20E06B03FCC0E0C3E58224FEF582E5CE
:105290008334FFF583D0E0C082C083E0FAA3E0FB53
:1052A000A3EAF0A3EBF0D083D082DCDAEE2456F54B
:1052B0008275830050020583787FE6F0A308E6F04C
:1052C0007900752F038F307531009000561203CD91
:1052D0001205671203CD12057B852F3285303312FC
:1052E0004CE4EFB583030252ED1F02521EC3227439
:1052F00009124E59D3221246ECF5831246ECF58280
:105300001246EC70101246EC700BAF371246EC6F81
:105310007003025318024914C01EC01F85831E85E6
:10532000821F1218817401F9747FF8752F0075308F
:105330000075310012046E787FE6C3951EC3951F79
:10534000D01FD01E251E251FF67401F9747FF87535
:105350002F0075300075310012041812472D0248D5
:10536000171246ECF583AF371246EC6F70A7128226
:105370002E12822E12822E124710E5361247057425
:1053800000124705E51A124705740012470574001C
:1053900012470574001247057400124705E53712DD
:1053A00047053099FD0248179053B0C082C0833240
:1053B0007581D475D0000261C2C082C083E58224A9
:1053C00020F582E583347DF5837401F9743BF8752B
:1053D0002F00858330858231120418D083D082C09B
:1053E00082C083E58275F008A42420F5825002056E
:1053F000F0A8F0E58375F008A4282400F583740470
:10540000F9747FF8752F0085833085823112041876
:10541000A3A3A3A37404F97483F8752F00858330C4
:10542000858231120418D083D082E5824583600ED4
:10543000E5822418E58334FC74FFF5F0500BC0823C
:10544000C083123B26D083D08222120941C0E0746F
:1054500001F9747FF8752F00753000753100120462
:105460006E787FE6D0F0C395F0F67401F9747FF89A
:10547000752F0075300075310012041822753B003D
:105480007854E4F2787F75F00876FF08D5F0FA22B8
:10549000751E30751F30C263C26475F005C0F0D24E
:1054A000A3C256C2A2D259D2A1C258D2A4C2571284
:1054B000547D12213DD0F0205009205106D5F0DD59
:1054C00002550712552C403F1200D77884E6B4FFEE
:1054D00005C32275F005C0F012213DD0F020510621
:1054E000D5F0F3025507E53CB4021C78A3E624F698
:1054F000401508E624F6400F78A3E62430F51E0890
:10550000E62430F51FC3221200ABD3227897797FAF
:105510007A05800678A379847A03E608540FC4F5E7
:10552000F0E608540F45F0F709DAEF222050313049
:10553000513AE53C600624FD24FC4030125514121B
:1055400000E475F005C0F0122139D0F02050112090
:105550004406D5F0F002556C1211F9B40B0E80031D
:1055600012550C753B007854E4F2C322D322222258
:10557000781DE254C07078E275F00A84C445F07872
:1055800081F6781CE254C07066E275F00A84C44566
:10559000F07882F6781BE254E07054E275F00A84E9
:1055A000C445F07883F6781AE2604454E07040E233
:1055B00075F00A84C445F0C0E07818E2030354C0D3
:1055C000D0F045F07884F67819E2602354F0701F2B
:1055D000E275F00A84C445F0C0E0781EE254F87029
:1055E0000EE2C42354E0D0F045F07885F6C322D310
:1055F0002290000075F019C0F07402F9747FF875FC
:105600002F0185833085823112046E7880B6FF02C7
:10561000801318E551300C0AB4FF0788F07855E282
:10562000A8F0666011E5822410F58250020583D04F
:10563000F0D5F0C3C322D0F0A3D322300C4DE582C5
:1056400024FFF582E58334FFF58375F019E58224A4
:1056500080E58334FE5005900000800AE582241026
:10566000F58250020583C0F07402F9747FF8752F3B
:105670000185833085823112046E7880B6FF028006
:105680000518E6B55107D0F0D5F0C2C322D0F0A37B
:10569000D322120114300C0C1255F1400390FFF18B
:1056A00012563B22C0511256C2D05122300C131256
:1056B00055F1400390FFF112563B5005F55112563B
:1056C000F422E55170057551108023B41005755111
:1056D00011801BB411057551208013B4200575513C
:1056E000FF800BB4FF0575510080037551FF125701
:1056F000A5E551222230130CC21312557040051239
:1057000064DE800312652C7884E6C45403E6540FEB
:105710007885E6C45401E6540F7883E6C4540FE656
:10572000540F7882E6C4540FE6540F22300C0A124C
:1057300055F150051256F480031257A522C2AC123F
:105740005FF4C2AC12822E12822ED299C2B674FFBE
:1057500012470575370074421247057462124705F7
:105760007415124705742A124705741B12470574F5
:1057700000124705740012470574001247057400B3
:105780001247051202FD75F010C0F07400124705B3
:10579000D0F0D5F0F4E5371247053099FDC24FD26D
:1057A000B6125FF42222201801227475787A120151
:1057B0002F501A206819D268125CAB7518C0751981
:1057C0000B741A543F4400F51A120A3722C26812A9
:1057D000652C203304203433227883E6543FF5F0DF
:1057E0007970E365F0702109E3788266701A2035DC
:1057F00016D235125CAB7518C075190B741A543F6C
:105800004400F51A120A372230342F7883E6543FC9
:10581000F5F07972E365F0702109E3788266701A19
:10582000203516D235125CAB7518C075190B741A79
:10583000543F4400F51A120A3722C23522C2AC1274
:105840000A75600CF5188819120DE0120A8D80EFA8
:10585000D2AC227E007F8490000075F000E4932596
:10586000F0F5F0A3C3E5829EE5839F40F0E5F0707C
:10587000022200E5F0C0E0E58312556FE582125583
:105880006FD0E012556FC2ADC2ACD21AD2A3C256CD
:10589000D2A2C259C2A1C258D2A4C257C2A080EC9F
:1058A000300C3C7400788A12013E40337F087E0041
:1058B0007478787A12012FCE13CE05E0DFF4201B26
:1058C0000E7400789A12013E5005EE655360108EFA
:1058D000538E517518C075190485511A120A372252
:1058E000C2AF75181075190FF51A120A37D2AF2208
:1058F00022300CFC205CF97401788A12013E40F0E1
:105900007477787A12012FE492E0C0E07476787AA6
:1059100012012FD0E033FE201B0E7401789A120181
:105920003E5005EE655460C88E54EE20E10630E02E
:105930002802596C30E014A25E725D50B3C25EC2A0
:105940005D125C0D74F81258E080A5D25EC25D1243
:105950005C0D74F71258E08097205D0ED25DC25E38
:10596000125C0DD25B74F61258E08084A22A825D2C
:1059700040F8D25DC25E125C2174F51258E0025804
:10598000F0C082C083D083D0822222304309C2A3D8
:10599000C256D2A4C25722D2A3C256C2A4C2572210
:1059A000200C0122300C19C0E0C082C083740712A1
:1059B0000188D083D082D0E040030259DE0259C072
:1059C000201B08206033D260205F2ED25FD260752A
:1059D00018C0751900751A0F120A370259F9201BE1
:1059E00008306015C260305F10C25FC2607518C0B9
:1059F000751900751A10120A37300C19C0E0C082F0
:105A0000C083740F120188D083D082D0E04003029B
:105A10005A33025A15201B08206233D26220612EAD
:105A2000D261D2627518C0751900751A51120A3701
:105A3000025A4E201B08306215C262306110C261EA
:105A4000C2627518C0751900751A52120A3722C23F
:105A5000B67537007403124705E51E124705E51FAA
:105A6000124705744E124705740812470574011257
:105A7000470574061247057848E2F5F0E5F012474D
:105A80000508E2F5F0E5F0124705784AE2F5F0E5A1
:105A9000F012470508E2F5F0E5F01247052442F858
:105AA000E2784CE2547FF5F07844E2C36001D3E53C
:105AB000F092E7F5F0E5F012470575F000E5F01219
:105AC0004705E5371247053099FD22C2B6126A35FF
:105AD0001269C47537007403124705E51E124705A5
:105AE000E51F124705744E124705740C12470574E2
:105AF00000124705740A124705C082C083A3A3A3FE
:105B0000E49375F064A4C0E0E5F0124705D0E0121C
:105B10004705A3A3A3A3E49375F064A4C0E0E5F054
:105B2000124705D0E0124705D083D082E493124794
:105B300005A3E493124705A3A3A3E493124705A387
:105B4000E493124705E58D124705E58B124705E5FD
:105B5000371247053099FD22C2B6121293C0E07584
:105B600037007403124705E51E124705E51F12476B
:105B700005744E1247057404124705740212470556
:105B80007402124705E57C124705D0F0E5F0124794
:105B900005E5371247053099FD22C2B6121213C02F
:105BA000E07537007403124705E51E124705E51F2F
:105BB000124705744E124705740412470574021209
:105BC00047057402124705E57C124705D0F0E5F061
:105BD000124705E5371247053099FD22C0F088F0DD
:105BE000C0F0C2AF7574007850E2F54BF5F008E2F2
:105BF000F54CD2AF45F0D0F0A8F0D0F07009B22A41
:105C0000202A04125C1722D22A75740322C2AF75AF
:105C10004BFF754CFFD2AF757400C20DC22AD2A7DC
:105C200022125BDCD25BD25522C26E026FA7D26E0B
:105C3000026FA7305D12202A0F543F4400F51A75F9
:105C400019087518C0120A3722D2B2C2B4D293C34F
:105C500022D2B2C2B4D29312821620B2ECC29312F4
:105C6000821630B2E4D29312821612821620B2D972
:105C7000C29312821612821630B2CED2B2C2B4D2FF
:105C800093D3221204B9C28474541204C4E41204DB
:105C9000931204A6F5F06448255D33F55DE5F02523
:105CA0005EB2E003F55ED9E9D284227583DD75F03A
:105CB00010752F03858330753100C083C0F0120347
:105CC000CD1208D3D0F0D0830583D5F0E47532FF30
:105CD0007533FF75750075760022E5822400C0E0FB
:105CE000E58334DDF8D0E0C322C082C0837401F9BB
:105CF000747FF8752F0385833085823112046E78A6
:105D00007FB6020CE57624FFF576E57534FFF57570
:105D1000D083D08222125CDAC082C083F58288836D
:105D2000125CE9787F76007401F9747FF8752F03AF
:105D3000858330858231120418D083D08222125C90
:105D4000DAC082C083F5828883C082C0837401F97F
:105D5000747FF8752F0385833085823112046E7845
:105D60007FB60209D083D082D083D08222E5762408
:105D700001F57650020575D083D082787F76027463
:105D800001F9747FF8752F03858330858231120401
:105D900018D083D08222125CDA125CDAC082C0830F
:105DA000F5828883125CE9787F76017401F9747F4B
:105DB000F8752F03858330858231120418D083D083
:105DC0008222125CDAC082C083F5828883125CE989
:105DD000787F76037401F9747FF8752F038583301B
:105DE000858231120418D083D08222125CDAC082FC
:105DF000C083F58288837401F9747FF8752F038559
:105E0000833085823112046E787FE6B40102800C03
:105E1000B402028007B4030280027400D083D082EF
:105E2000221204B9C28474541204C4E412049312FA
:105E300004A6B40205755D018002D9F3D2842275EF
:105E40005D007583DD75F00F752F03858330753127
:105E500000C083C0F01203CD1204DD1203CD79001F
:105E6000125E21D0F0D0830583E55D7026D5F0D891
:105E7000752F038583307531001203CD1204DD12B6
:105E800003CD79A0125E217532FF7533FFE55D7099
:105E900002D322C322E576457560167867E2F5F0F5
:105EA00008E245F0600BD37868E2957618E29575C4
:105EB00022C322C28C758A45758C5DD28CB20020BB
:105EC000000132C000C001C0D0C0E0C0F075D008F1
:105ED000D2541211F8125FD5051DE51D20E00C20EB
:105EE000E109301A1AE51D541F6059201A04E54AC9
:105EF0006002B2B5D0F0D0E0D0D0D001D0003220D6
:105F00005905A22AB392A2E51D30E203126D03E502
:105F10001D541F7032D255C27278ABE2D5E006D262
:105F200071D272743CF2C082C083126BD6D083D01F
:105F300082E4B54648B5485AB56262B56D63B57D31
:105F400067B57E68B54969E4B54A43B54771B5445C
:105F500072B54D76B57477E54C454B601DE54C2424
:105F600001F54C5002054B454B700FC20D205C0AE9
:105F7000205D07125C17D25BD255025EEBD546B5A9
:105F8000C20D7548B4757B00D247D24A80A7154A26
:105F900080B9D548A3C245C246C247809B156280DE
:105FA0009AD56D9AC2708096157D8095157E8094E5
:105FB000D54994754503301A030253A8025F38157A
:105FC00047808BD5448BD24E8087154D8086D57403
:105FD00086C2A78082E51DA2E330560292A3305903
:105FE0000292A230580292A122C2B6204F02D2B62B
:105FF000125FF43275C800C2ADC2AC75CBFF75CA72
:106000009875CDFF75CC98759853C298C299D2AC4B
:10601000C2BC75C8347599062275C800C2ACC2AD41
:1060200075980075CC2B75CDEBD2AD75C804227573
:10603000C800C2ACC2AD759800E58A242BF5CC54DB
:106040000F658C24EBF5CDD2AD75C80422C2A8C271
:10605000AAC289C28BC2ACC2A9C2AB758F0112059C
:10606000BCD21A125C2E125C0DE4F53B7854F27827
:106070007A75F010F2D5F0FCC25CC25DC25EC25F00
:10608000C261753DFF753FFF751D04C244C245C224
:1060900046C247754801754900C24AD2547571001D
:1060A000C235C21CC21DD24EC24F754410E4F54029
:1060B000F541F542F534F536121EB6751E00751F12
:1060C00080E4F546F54FF54EF557F558F53EC227F5
:1060D000C228C229C2037437785AF2785BF2785C1E
:1060E000F2785DF2D22375450375470178AB7A05E6
:1060F00076FF08DAFBC2137818E47A07F208DAFCB4
:10610000C2147551FF855153C215C20C757D0375BC
:10611000621E756300C267C211C212C20DC20EC2F6
:106120000FC263C264756000755F0075F006784247
:10613000E4F208D5F0FB7948E4F309F3794AF3096E
:10614000F3784CE4F2121407754AFAB2B57532FFCF
:106150007533FFD268756C007827740AF2126A14DE
:10616000C270756D0175701AC208C209C205C206F7
:10617000C207D2A075740075750075760078AA7490
:10618000FAF2E478B2F278B3F278B4F278AB743C15
:10619000F2C274C273C26F757B00126B49C275D2B2
:1061A00076C277758901758A3E758C5DC2B9D2A9B0
:1061B000D28CD2B6125FF4D2AFD293C2B4D2B2B202
:1061C000B522C21A75500375F0031281FED5F0FA9C
:1061D000C263C26412241D75500375F0031281FE60
:1061E000D5F0FAC263C2641222BCC2AF0200002022
:1061F000071320060820090D200802C32212141BD1
:1062000012661FD322126728D32275F000C0F01245
:106210007186D0F0500343F008E5F022307314206B
:10622000432278B4E2307106C271600214F224FA9B
:1062300050092230740E78B4E27009E57A54017086
:10624000031200E422C274C273E478B4F222C2AF33
:10625000754AFAB2B5128216B2B5128216B2B5D22A
:10626000A07581D475D00012604D12598112585317
:10627000125CAB121CDF754AFA120CDE1261EF756C
:1062800050031225971225AD1200F175188075196B
:1062900004751A80120A37D21B300C0F120B04122D
:1062A00058A01258F11257A61259A0D2B7D2AFC2B5
:1062B0001AC21B00000020B70912821620B7030281
:1062C0001CF9300C32120B0412621CE57854206069
:1062D0001178AAE2D5E00A12652C12573D78AA740B
:1062E000FAF2E57B6002157B300C0C1258A01258B4
:1062F000F11257A61259A0E5636003D5630E126B25
:10630000421226911256F512572C800CD2A3C25677
:10631000C2A1D258D2A4C257E562700312583DC23E
:1063200059D2A1C25812598BC263C264D25B786041
:10633000E2600D24FD40097573021227801261EF9F
:106340007861E2600D24FD40097573031227801205
:1063500061EFE5775440600620A803128101122105
:106360003D205108205005205202801A302F09305C
:10637000460612598102637E1233181261EF7827A4
:10638000E215E0F2700878277414F20262AB026240
:10639000E20074A2126426E8126461E912646112D8
:1063A00064982274A2126426E8126461E7126461A0
:1063B00009D582F81264982274A2126426E8126445
:1063C0006174A3126426126481F709D582041264F1
:1063D0009822C296D297000000C29780E974A21258
:1063E0006426E81264611263EA2274A3126426121E
:1063F0006481F91264982274A27A08C2960000009F
:10640000C297335005D29602640CC296D297000010
:1064100000C297DAEDD29600D297000000309604C1
:10642000C297C322D3227A08D296D29700000000E6
:10643000000000000000000000000000C296000004
:1064400000C297335005D29602644DC296D297008F
:106450000000C297DAEDD29600D297000000C297F2
:10646000227A08335005D29602646DC296D2970004
:106470000000C297DAEDD29600D297000000C297D2
:10648000227A08D296C29700000000D297C33096B5
:1064900001B333DAF0C29722C296000000D297000F
:1064A0000000D29622781079D0C0827582051263DE
:1064B000B8D08278D0B6870E08B6E00A08B63306A0
:1064C00008B6A902C322D3221264A5400122788112
:1064D0007600087600087600087601087601787F55
:1064E00076000876007883E6543FF67800797FC01E
:1064F000827582071263A3D0821281FE7814797F9D
:10650000C0827582071263A3D0821281FE78D07692
:10651000870876E00876330876A9781079D0C082AB
:106520007582041263A3D0821281FE2278027981DF
:10653000C0827582051263B8D082227885E603C4D2
:10654000540775F018A4C0E07883E6C4540375F0CE
:106550000AA4F5F0E6540F25F0D0F025F075F03CD4
:10656000A4C0F0C0E07882E6C4540775F00AA4F530
:10657000F0E6540F25F0D0F025F0F5F0D0E034002F
:10658000C5F022207556206921C0D0C0E0E8C0E0E7
:10659000C0F0E54D700385706E754D08D26C1266C3
:1065A0009BD0F0D0E0F8D0E0D0D0C2893220692969
:1065B000C0D0C0E0E8C0E0C0F0E54D7003756E00EB
:1065C000754D08A2B2B3926C126780308502D20575
:1065D000D0F0D0E0F8D0E0D0D0C28B32C2A8C289CF
:1065E000322075C9206926C0D0C0E0E8C0E0C0F004
:1065F000E54D700385706E754D08C26C12669B3058
:106600008502D205D0F0D0E0F8D0E0D0D0C28B32F5
:10661000C2A8C2AAC293C2B4C0E01281FED0E0C236
:1066200075C293C2B4C289C28BD2B2D2B3C26975E9
:106630004D0085706EC205C2B8D288D2A8C2BAD247
:106640008AD2AA22C275C2A8C2AAC289C28B22E576
:1066500070141475F00884F5F0C0F0782EE230E084
:1066600002B26A30E102B26A30E202B26A30E30298
:10667000B26A08D5F0E7D0F0E230E002B26B30E168
:1066800002B26B30E202B26B30E302B26B08D5F0BB
:10669000E7206A05306B02C322D322E56EB570078E
:1066A000A26C926A0266E5B40107A26C926B026664
:1066B000E5C3E57014956E403275F00484242EF81D
:1066C000E205F0D5F006A26C92E38016D5F006A2A2
:1066D0006C92E2800DD5F006A26C92E18004A26C6F
:1066E00092E0540FF2D56E02D2692285706ED269A3
:1066F00022754732126610305405C25412027AE5F0
:106700004760113069F1E56E700A12664412664FF7
:106710004002C322126644D322C2A8C2AAC293C2B4
:10672000B4C0E01281FED0E0D275C293C2B4C28977
:10673000C28BD2B2D2B3C269754D00756E00C2056C
:10674000C2BAD28AD2AA22754732126719305405CA
:10675000C25412027AE547600C3069F1E56E7005AB
:10676000126644C322126644D322C330E001B33020
:10677000E101B330E201B330E301B330E401B3220D
:10678000E56E75F00584C0E024ECD0E04055242E81
:10679000F8E2A26C92E503F2E56E700BE2541FB4CE
:1067A0000B40756E05803B056EE5F0B40434E212D3
:1067B000676A502F540FF218E2540FB40F24D3E835
:1067C000942E782EF20404C082F58275F00B08E254
:1067D00065F0F5F0D582F7D082540F7006D2697556
:1067E0006E00221267282201000000000000000055
:1067F000000A000000000000000000040600000085
:106800000000000000080E0300000000000000006F
:10681000010702000000000000000A060801000055
:10682000000000000402040F000000000000080641
:10683000090809000000000000010E050F05000016
:106840000000000A0C0A090B0300000000040E0BF4
:1068500000040502000000080E06070804070100F6
:10686000000001050A040D080E75F00A79977700FB
:1068700009D5F0FA782EE2FA60400824F25007EACF
:1068800024F328F87A0DE2540FF26029EA1475F027
:106890000AA424E7F58274003467F58379A07E00AA
:1068A0007B0AE493F5F0E2A42E2775F01084FEA78E
:1068B000F0A319DBED08DACEC322D322094300A0EE
:1068C0000954009F0966009E0977009D0989009C74
:1068D000099B009B09AD009A09BF009909D2009855
:1068E00009E4009709F700960A0A00950A1D00942A
:1068F0000A3000930A4300920A5700910A6B0090F5
:106900000A7F008F0A93008E0AA7008D0ABB008CB5
:106910000AD1008B0AE7008A0AFE00890B1400885E
:106920000B2B00870B4300860B5C00850B750084E6
:106930000B8E00830BA700820BC100810BDB008054
:106940000BF6007F0C10007E0C2B007D0C47007CAA
:106950000C64007B0C81007A0C9E00790CBB0078E3
:106960000CDB00770CFB00760D1B00750D3B0074F3
:106970000D5B00730D7D00720D9F00710DC20070E4
:106980000DE4006F0E07006E0E2C006D0E51006CB2
:106990000E76006B0E9B006A0EC100690EE900685E
:1069A0000F1100670F3900660F6100650F890064E1
:1069B0000FB300630FDE0062100900611034006045
:1069C000105F005F7F429068BCE493A3F5F0E4930E
:1069D000A3C3958BE5F0958D5015A3A3DFEBE5825E
:1069E00024FFF582E58334FFF583E49314800BA341
:1069F000E493BF42059068BC8010C0E0E58224F9B2
:106A0000F582E58334FFF583D0E02290006BE0A2AD
:106A10008733F02290006C7400F090006B7455F096
:106A200090006D74FFF090006F7405F090006E742C
:106A300012F0D28122D286A2A4C0D0D2A475F000D6
:106A4000D5F0FDD5F0FDC28E53890F438910758BAB
:106A500000758D00C28FC2AFC2A4D28E20860330D3
:106A60008FFAC28E308F06758BFF758DFFD2AFD037
:106A7000D092A422F024FE4005308102C2812290EF
:106A8000006FE0D5E0EE7442F0126A35D281E58BFA
:106A90002499E58D34F24014E58B24E1E58D34F33F
:106AA000400EE58B24E0E58D34FC4008741580062B
:106AB000741180027412FE90006EE06E6013EEF0AE
:106AC000E5775404700B7518C07519008E1A120AF8
:106AD0003722126A0B603904603690006DE020E0C6
:106AE00010D2E0F090006CE070047405F022E4F045
:106AF0002290006CE0602C14F07028E5775402704E
:106B0000227518C0751900751A14120A37026B2302
:106B100090006DE030E00DC2E0F090006CE070CECF
:106B2000743CF02290006CE060F914F070F5E577A9
:106B3000540270EF7518C0751900751A13120A37D0
:106B400080E1126A7F126AD2229002EC75F008E4AA
:106B5000F0A3D5F0FB9002F475F00874FFF0A3D514
:106B6000F0FB22C0E0126BB6D0E0B3502CC0E024A2
:106B7000F8D0E04022C082C083F5F024F4F582E42E
:106B80003402F583E0C5F024ECF582E43402F583A9
:106B9000E5F0F0D083D082D322C0E024F8D0E040EA
:106BA00013C082C08324ECF582E43402F583E4F060
:106BB000D083D082C322C0E024F8D0E04016C08247
:106BC000C08324ECF582E43402F583E0D083D082E4
:106BD0006002D322C3229002EC75F008E06003B497
:106BE000FF05A3D5F0F62220E70414F080F43072FC
:106BF000F114F0B480ECE4F080E8B44007740012C3
:106C00006BB6803DB441077401126BB68033B44259
:106C1000077402126BB68029B443077403126BB673
:106C2000801FB444077404126BB68015C0E024E4DE
:106C3000D0E040132324B0C0E07400346CC0E022E4
:106C4000C3740122D380FAE4C322A243B380F2D2F8
:106C500055A26F80EC80F0A20D80E6A20F80E2A228
:106C60007780DE80DF80E0A20E80D63070D280D4C4
:106C7000E575457660CA80CC125E9580C4A25E72CE
:106C80005DB380BDA25D822A80B7A25DB02A80B1CB
:106C9000A25E80ADC330730920430678B4E2700170
:106CA000D3809EA26EB38099C3E57D6001D38091AD
:106CB0008098809B80998097809580938091808F29
:106CC0008093809380958097809980998099809B0C
:106CD000809E80A480A780AC80B080B480B680C342
:106CE00080C68004800E8018C3204305E57E6001C5
:106CF000D3026C41C3304305E57E6001D3026C4191
:106D0000026C47126DFD300C19C0E0C082C0837464
:106D100004120188D083D082D0E04003026D380293
:106D20006D22E538B40D0A302502802CD225D3809F
:106D300015126BFA6022800EE538B40D062025038B
:106D4000026D58C225C34009C22BA22BB392A58065
:106D500007D22BA22BB392A5300C19C0E0C082C081
:106D6000837405120188D083D082D0E04003026D85
:106D70008A026D74E539B40D0A302602802CD226C1
:106D8000D38015126BFA6022800EE539B40D06200F
:106D90002603026DAAC226C34009C22CA22CB392BC
:106DA000A68007D22CA22CB392A6300C19C0E0C04A
:106DB00082C083740B120188D083D082D0E040035C
:106DC000026DDC026DC6E53AB40D0A300202802C79
:106DD000D202D38015126BFA6022800EE53AB40D10
:106DE00006200203026DFCC202C34009C204A204D1
:106DF000B392808007D204A204B3928022B21030F2
:106E00001060E5785410600330431BE5795404703A
:106E100003204538E57954017003204611E5795483
:106E2000027003204717C26F754F00026E62E54F74
:106E3000B401028024754F01754E40801CE54FB4AB
:106E400002028015754F02754EA0800DE54FB40308
:106E5000028006754F03754EF0E54E23F54EA2E015
:106E6000926F22C22BA22BB392A522D22BA22BB3BC
:106E700092A522B22BA22BB392A522F5F0030354C4
:106E80003FB40258E53864086005E538B40D4AE5BA
:106E9000F089F0C0F0300C19C0E0C082C0837404E7
:106EA000120188D083D082D0E04003026EC0026E0F
:106EB000B1D0F0A9F05403B4020D126E63026FA5B5
:106EC000D0F0A9F0026FA5B40106126E6B026FA597
:106ED000B40306126E73026FA5026FA3B40362E5DA
:106EE0003964086005E539B40DEFE5F089F0C0F0CC
:106EF000300C19C0E0C082C0837405120188D083B1
:106F0000D082D0E04003026F1F026F0CD0F0A9F0D6
:106F10005403B40211C22CA22CB392A6026FA5D0C6
:106F2000F0A9F0026FA5B4010AD22CA22CB392A64C
:106F3000026FA5B40309B22CA22CB392A68066807E
:106F400062B4045FE53A64086005E53AB40D54E5BF
:106F5000F089F0C0F0300C19C0E0C082C083740B1F
:106F6000120188D083D082D0E04003026F83026F89
:106F700071D0F0A9F05403B4020FC204A204B3927A
:106F8000808022D0F0A9F0801CB40109D204A204B0
:106F9000B392808010B40309B204A204B39280803B
:106FA000048000D322C322C0E07417306E21B538AC
:106FB00007C22BA22BB392A5B53907C22CA22CB3C2
:106FC00092A6B53A07C204A204B39280D0E022B5DB
:106FD0003807D22BA22BB392A5B53907D22CA22CFD
:106FE000B392A6B53A07D204A204B39280D0E022AD
:106FF000C0E0127173D0E04021302E0320431B20EB
:107000005E18C0E0125C33125C21D0E0203A091215
:1070100081A7751810120A37D322203A091281A7C6
:10702000751820120A37C322D20F7518C0751900BF
:10703000751A01120A37302A19205D1C20380DC23A
:10704000AF754BFF754CF8D2AF125C177852E2F572
:1070500046222036031270F622E51A543F44C0F54A
:107060001A751908C25EC25D205C46125C0DD25BC7
:10707000803FE51A543F4480F51A751908D25E80A6
:10708000E5E51A543F4440F51A751908D25DC25E11
:10709000205C1E125C0DD25B8017E51A543F440041
:1070A000F51A751908D25DC25E8000205C03125C7F
:1070B000217518C0120A372230190122C0E074105D
:1070C0008004C0E0741178A3760A0875F00A84F68B
:1070D00008A6F0753C03D0E078AEF2087405F2D251
:1070E0001922C20F754600C2477518C07519007580
:1070F0001A02120A3722757B00D2457548B47518FA
:107100005075190F751AFF120A3722751860751914
:107110000F751AFF120A37757E03C245C2482275E1
:10712000187075190F751AFF120A37757E0322122F
:107130005CABE51A543F4400F51A75190B7518C07D
:10714000120A37227874F208F21226617518C07597
:107150001900751A50120A3722400C305C08C25CC4
:10716000205D03125C0D22205CFC125C33125C215A
:10717000D25C221274AA400D1278654008127C205D
:107180004003127FDE221274B5400D127870400861
:10719000127C2B4003127FE922A290302001B378A9
:1071A0005AE233F222107603027553301A08C3787C
:1071B0005AE4F20274C3E579541060033043EF7867
:1071C0005AE260EF04600302755120230320274D2B
:1071D000D227300C19C0E0C082C08374001201882D
:1071E000D083D082D0E040030275510271EE785610
:1071F000E224B0401CC082C083907408E225E00401
:1072000093F5F0E225E093D083D082C0F0C0E0E2B5
:1072100022E2751890751909F51A120A370275518C
:1072200012598B1200D70275517401127028027521
:10723000517401126FF040E8027551C24312710B94
:10724000027551D270756D05027212C0E0740112A0
:107250006B6DD0E002721220430320370CC0E07443
:1072600004126B6DD0E0027212027551743D02730C
:1072700035027212C0E0E57A54047005D0E0027263
:1072800012D0E0027551C0E0D37401127159D0E000
:1072900002721202721202721274001270B8027537
:1072A0005174101270B802755174111270B80275D1
:1072B0005174201270B80275517401F9747FF87519
:1072C0002F0075308C7531F112046E787FE61270E4
:1072D000B80275517401F9747FF8752F0075308C00
:1072E0007531F112046E787FE61270C2027551306A
:1072F000741C78B3E2601778B4F27518C075190978
:107300007401543F4480F51A120A37027220027544
:10731000513074FAE478B4F27518C0751909740123
:10732000543F4440F51A120A37027220751A0112AE
:10733000712F027220204308D24312711F02722063
:10734000C24312710B027220E57754106007E412F9
:107350007144027220027551E5775410600874FF81
:10736000127144027220027551751A01127059028D
:107370007551751A0112709A027551751A011270C1
:1073800081027551751A01127072027551740012E2
:107390006B6D740112824A0272207400126B997430
:1073A000011282590272207400126BB640EC027313
:1073B0008D7402126B6D7401128268027220740265
:1073C000126B9974011282770272207402126BB6EA
:1073D00040EC0273B17403126B6D74011282860269
:1073E00072207403126B99740112829502722074D8
:1073F00003126BB640EC0273D530430302734002B4
:1074000075512043FA027338755172297231723BFB
:107410007212721272127243724B7257726C721243
:107420007271727472867212721272127212721207
:10743000721272127212721272127212721272122C
:10744000721272127212721272127212721272121C
:10745000721272127212721272127212721272120C
:1074600072127212721272127212721272937296F7
:10747000729972A172A972B172B972D472EF73115A
:10748000732C73357348735873697372737B738489
:10749000738D739A73A773B173BE73CB73D573E295
:1074A00073EF721273F9740272127856E2B40B031E
:1074B000A22722C3222043097856E2B40D03A22753
:1074C00022C322202306202703027551C227300C35
:1074D00019C0E0C082C0837400120188D083D082BA
:1074E000D0E040030275510274EA7856E260DAB4E3
:1074F00001061270E2027551B40203027551B40321
:1075000007D24312711F8049B4090820433630372F
:1075100033803EB40A02743DB40D0BE57A54047016
:1075200030740D027544B40E0BC37401127159749A
:107530000E027544C0E024CED0E05008C0E024B074
:10754000D0E0500D7518A0751909F51A120A378088
:1075500000D27622A291302101B3785BE233F2228D
:1075600010760302790E301A08C3785BE4F20278D1
:107570007EE579542060033043EF785BE260EF04EE
:10758000600302790C20230320284DD228300C19E7
:10759000C0E0C082C0837401120188D083D082D041
:1075A000E0400302790C0275A97857E224B0401C30
:1075B000C082C0839077C3E225E00493F5F0E22512
:1075C000E093D083D082C0F0C0E0E222E275189050
:1075D00075190AF51A120A3702790C12598B120022
:1075E000D702790C740212702802790C7402126F9F
:1075F000F040E802790CC24312710B02790CD27090
:10760000756D050275CDC0E07401126B6DD0E0029E
:1076100075CD20430320370CC0E07404126B6DD08D
:10762000E00275CD02790C743D0276F00275CDC092
:10763000E0E57A54047005D0E00275CDD0E002791F
:107640000CC0E0D37402127159D0E00275CD0275FE
:10765000CD0275CD74001270B802790C74101270DE
:10766000B802790C74111270B802790C742012707F
:10767000B802790C7401F9747FF8752F0075308C9D
:107680007531F512046E787FE61270B802790C74C9
:1076900001F9747FF8752F0075308C7531F512047F
:1076A0006E787FE61270C202790C30741C78B3E2F7
:1076B000601778B4F27518C07519097402543F4404
:1076C00080F51A120A370275DB02790C3074FAE47D
:1076D00078B4F27518C07519097402543F4440F526
:1076E0001A120A370275DB751A0212712F0275DB46
:1076F000204308D24312711F0275DBC24312710B83
:107700000275DBE57754106007E41271440275DB03
:1077100002790CE5775410600874FF127144027509
:10772000DB02790C751A0212705902790C751A0273
:1077300012709A02790C751A0212708102790C7516
:107740001A0212707202790C7400126B6D740212BC
:10775000824A0275DB7400126B997402128259021C
:1077600075DB7400126BB640EC0277487402126B42
:107770006D74021282680275DB7402126B997402D6
:107780001282770275DB7402126BB640EC02776CE2
:107790007403126B6D74021282860275DB7403121D
:1077A0006B9974021282950275DB7403126BB640FA
:1077B000EC0277903043030276FB02790C2043FA07
:1077C0000276F3790C75E475EC75F675CD75CD75AB
:1077D000CD75FE76067612762775CD762C762F76C9
:1077E0004175CD75CD75CD75CD75CD75CD75CD7515
:1077F000CD75CD75CD75CD75CD75CD75CD75CD7579
:10780000CD75CD75CD75CD75CD75CD75CD75CD7568
:10781000CD75CD75CD75CD75CD75CD75CD75CD7558
:10782000CD75CD75CD75CD764E76517654765C7628
:1078300064766C7674768F76AA76CC76E776F07777
:107840000377137724772D7736773F774877557707
:1078500062776C777977867790779D77AA75CD7701
:10786000B477BD75CD7857E2B40B03A22822C322AA
:107870002043097857E2B40D03A22822C322202313
:107880000620280302790CC228300C19C0E0C082FF
:10789000C0837401120188D083D082D0E0400302FB
:1078A000790C0278A57857E260DAB401061270E22A
:1078B00002790CB4020302790CB40307D2431271AB
:1078C0001F8049B40908204336303733803EB40A5C
:1078D00002743DB40D0BE57A54047030740D0278D7
:1078E000FFB40E0BC37402127159740E0278FFC0FC
:1078F000E024CED0E05008C0E024B0D0E0500D75B8
:1079000018A075190AF51A120A378000D27622A239
:1079100092302201B3785CE233F222107603027CCB
:10792000C9301A08C3785CE4F2027C39E579544026
:1079300060033043EF785CE260EF046003027CC7D1
:1079400020230320294DD229300C19C0E0C082C069
:10795000837402120188D083D082D0E04003027C7D
:10796000C70279647858E224B0401CC082C083907A
:107970007B7EE225E00493F5F0E225E093D083D00E
:1079800082C0F0C0E0E222E275189075190CF51A79
:10799000120A37027CC712598B1200D7027CC774B7
:1079A00003127028027CC77403126FF040E8027C57
:1079B000C7C24312710B027CC7D270756D05027984
:1079C00088C0E07401126B6DD0E002798820430317
:1079D00020370CC0E07404126B6DD0E0027988028D
:1079E0007CC7743D027AAB027988C0E0E57A540422
:1079F0007005D0E0027988D0E0027CC7C0E0D37483
:107A000003127159D0E0027988027988027988746A
:107A1000001270B8027CC774101270B8027CC77470
:107A2000111270B8027CC774201270B8027CC7743F
:107A300001F9747FF8752F0075308C7531F71204D9
:107A40006E787FE61270B8027CC77401F9747FF813
:107A5000752F0075308C7531F712046E787FE61241
:107A600070C2027CC730741C78B3E2601778B4F23D
:107A70007518C07519097403543F4480F51A120A29
:107A800037027996027CC73074FAE478B4F275183C
:107A9000C07519097403543F4440F51A120A37029D
:107AA0007996751A0312712F027996204308D243F2
:107AB00012711F027996C24312710B027996E57713
:107AC00054106007E4127144027996027CC7E5778E
:107AD0005410600874FF127144027996027CC775D5
:107AE0001A03127059027CC7751A0312709A027C2D
:107AF000C7751A03127081027CC7751A031270725F
:107B0000027CC77400126B6D740312824A0279966C
:107B10007400126B997403128259027996740012E0
:107B20006BB640EC027B037402126B6D740312821D
:107B3000680279967402126B997403128277027943
:107B4000967402126BB640EC027B277403126B6DC5
:107B500074031282860279967403126B997403126D
:107B600082950279967403126BB640EC027B4B301F
:107B70004303027AB6027CC72043FA027AAE7CC77E
:107B8000799F79A779B179887988798879B979C124
:107B900079CD79E2798879E779EA79FC7988798809
:107BA00079887988798879887988798879887988CD
:107BB00079887988798879887988798879887988BD
:107BC00079887988798879887988798879887988AD
:107BD000798879887988798879887988798879889D
:107BE00079887A097A0C7A0F7A177A1F7A277A2F8E
:107BF0007A4A7A657A877AA27AAB7ABE7ACE7ADFC7
:107C00007AE87AF17AFA7B037B107B1D7B277B3441
:107C10007B417B4B7B587B6579887B6F7B78798850
:107C20007858E2B40B03A22922C3222043097858D2
:107C3000E2B40D03A22922C3222023062029030235
:107C40007CC7C229300C19C0E0C082C08374021204
:107C50000188D083D082D0E04003027CC7027C60E0
:107C60007858E260DAB401061270E2027CC7B4020E
:107C700003027CC7B40307D24312711F8049B409C1
:107C800008204336303733803EB40A02743DB40DC9
:107C90000BE57A54047030740D027CBAB40E0BC339
:107CA0007403127159740E027CBAC0E024CED0E085
:107CB0005008C0E024B0D0E0500D7518A075190C24
:107CC000F51A120A378000D27622A285300101B35C
:107CD000785DE233F22210760302808C301A08C3FA
:107CE000785DE4F2027FF7E579548060033043EF7A
:107CF000785DE260EF04600302808A2023032003A2
:107D00004DD203300C19C0E0C082C083740A120146
:107D100088D083D082D0E0400302808A027D1F7821
:107D200059E224B0401CC082C083907F3CE225E031
:107D30000493F5F0E225E093D083D082C0F0C0E058
:107D4000E222E275189075190DF51A120A370280B1
:107D50008A12598B1200D702808A7404127028028A
:107D6000808A7404126FF040E802808AC243127164
:107D70000B02808AD270756D05027D43C0E07401EC
:107D8000126B6DD0E0027D4320430320370CC0E02E
:107D90007404126B6DD0E0027D4302808A743D0250
:107DA0007E6902808A027D43C0E0E57A5404700552
:107DB000D0E0027D43D0E002808AC0E0D374041298
:107DC0007159D0E0027D43027D43027D437400126D
:107DD00070B802808A74101270B802808A7411120E
:107DE00070B802808A74201270B802808A7401F917
:107DF000747FF8752F0075308C7531F312046E782E
:107E00007FE61270B802808A7401F9747FF8752FCA
:107E10000075308C7531F312046E787FE61270C2F3
:107E200002808A30741C78B3E2601778B4F2751857
:107E3000C07519097404543F4480F51A120A3702B8
:107E40007D5102808A3074FAE478B4F27518C075F6
:107E500019097404543F4440F51A120A37027D513F
:107E6000751A0412712F027D51204308D2431271FA
:107E70001F027D51C24312710B027D51E5775410F0
:107E80006007E4127144027D5102808AE577541044
:107E9000600874FF127144027D5102808A751A04D1
:107EA00012705902808A751A0412709A02808A75BB
:107EB0001A0412708102808A751A0412707202808C
:107EC0008A7400126B6D740412824A027D51740030
:107ED000126B997404128259027D517400126BB6B0
:107EE00040EC027EC17402126B6D7404128268024F
:107EF0007D517402126B997404128277027D517461
:107F000002126BB640EC027EE57403126B6D7404D2
:107F1000128286027D517403126B99740412829549
:107F2000027D517403126BB640EC027F09304303AB
:107F3000027E7402808A2043FA027E6C808A7D5A17
:107F40007D627D6C7D437D437D437D747D7C7D883A
:107F50007D9D7D437DA27DA87DBA7D437D437D438C
:107F60007D437D437D437D437D437D437D437D4311
:107F70007D437D437D437D437D437D437D437D4301
:107F80007D437D437D437D437D437D437D437D43F1
:107F90007D437D437D437D437D437D437D437D43E1
:107FA0007DC77DCA7DCD7DD57DDD7DE57DED7E08FE
:107FB0007E237E457E607E697E7C7E8C7E9D7EA655
:107FC0007EAF7EB87EC17ECE7EDB7EE57EF27EFF1A
:107FD0007F097F167F237D437F2D7F367D43785930
:107FE000E2B40B03A20322C3222043097859E2B46E
:107FF0000D03A20322C32220230620030302808A4A
:10800000C203300C19C0E0C082C083740A12018818
:10801000D083D082D0E0400302808A02801E78594B
:10802000E260DAB401061270E202808AB40203024E
:10803000808AB40307D24312711F804EB40908200E
:10804000433B3037388043B40A02743DB40C02809D
:1080500039B40D0BE57A54047030740D02807DB490
:108060000E0BC37404127159740E02807DC0E0249B
:10807000CED0E05008C0E024B0D0E0500D7518A07C
:1080800075190DF51A120A378000D27622E5775459
:1080900040601AE578540270061271991271A5E5D4
:1080A0007854047006127554127560800C12719920
:1080B0001271A512755412756012790F12791B1284
:1080C0007CCA127CD6C223204A0122C24A7518C03B
:1080D000751900751A54120A3722E8C0E07856E282
:1080E000640360187857E2640360117858E264030F
:1080F000600A7859E264036003C38001D3D0E0F8DA
:1081000022E4A22A92E0A22B92E1A22C92E2A20403
:1081100092E3F5727573051225D774035004122784
:108120005D221227377890E6C0E0E57854026012AD
:10813000D0E0C0E0540712815FD0E0C0E0540712E5
:10814000815FE57854046014D0E0C0E0C4540712A5
:108150008183D0E0C0E0C45407128183D0E022A222
:1081600027302001B34007D320E10A028182C320D7
:10817000E203028182302001B3E49400785AF212C3
:1081800071A522A228302101B34007D320E10A02C1
:1081900081A6C320E2030281A6302101B3E494004A
:1081A000785BF212756022B4010775190F751AE138
:1081B00022B4020775190F751AE222B40307751964
:1081C0000F751AE322B4040775190F751AE422B467
:1081D000110775190F751AD122B4120775190F7589
:1081E0001AD222B4130775190F751AD322B41407C3
:1081F00075190F751AD42275190F751AD422C28EEB
:1082000053890F438910758BD6758D97C28FD28E87
:10821000308FFDC28E22C28E53890F438910758B19
:10822000EB758DCBC28FD28E308FFDC28E22C28E67
:1082300053890F438910E58AC4242BF58B758DEB88
:10824000C28FD28E308FFDC28E22543F4400F51A69
:1082500075190A7518C0020A37543F4480F51A751B
:10826000190A7518C0020A37543F4400F51A7519E7
:108270000C7518C0020A37543F4440F51A75190CA2
:108280007518C0020A37543F4480F51A75190C75E9
:1082900018C0020A37543F44C0F51A75190C7518F6
:1082A000C0020A377401126B997404126B99220090
:1082B00000000000000000000000000000000000BE
:1082C00000000000000000000000000000000000AE
:1082D000000000000000000000000000000000009E
:1082E000000000000000000000000000000000008E
:1082F000000000000000000000000000000000007E
:10830000000000000000000000000000000000006D
:10831000000000000000000000000000000000005D
:10832000000000000000000000000000000000004D
:10833000000000000000000000000000000000003D
:10834000000000000000000000000000000000002D
:10835000000000000000000000000000000000001D
:10836000000000000000000000000000000000000D
:1083700000000000000000000000000000000000FD
:1083800000000000000000000000000000000000ED
:1083900000000000000000000000000000000000DD
:1083A00000000000000000000000000000000000CD
:1083B00000000000000000000000000000000000BD
:1083C000000000000000000000000000000050520B
:1083D000343032207665722E3132382E342E3220EF
:1083E0004864773A482030322D30382D30352030EF
:1083F000303A31332020004352430000000000ADEA
:00000001FF
:0300000306028072
